:020000040000FA
:10000000F26A72EF01F0FFFF78EF13F0FFFFFFFFDE
:10001000FFFFFFFFFFFFFFFF7AEF13F0A96EA69E21
:10002000A69CA680A8501200A86EA69EA69CA68498
:10003000F29EF2BE18EF00F0550EA76EAA0EA76E44
:10004000A682F28EA6941200C70ED56E940ED66EBE
:10005000F294F2A429EF00F0120024EC00F024EC5A
:1000600000F024EC00F024EC00F024EC00F024EC90
:1000700000F024EC00F024EC00F024EC00F024EC80
:1000800000F012002DEC00F02DEC00F02DEC00F053
:100090002DEC00F02DEC00F02DEC00F02DEC00F03C
:1000A0002DEC00F02DEC00F02DEC00F0120052ECE5
:1000B00000F037EC00F01200150EA96EFF0E14ECE4
:1000C00000F024EC00F01200150EA96E5A0E14EC8C
:1000D00000F024EC00F01200A68EF86A000EF76E15
:1000E000000EF66EFE0E606F3F0E616FED0E626FDA
:1000F000DE0E636F0900F550631B0900F550621BAB
:10010000020E605F000E615B60516111D8A47AEF4E
:1001100000F0621F631F0900F550635DD8A4A2EFD1
:1001200000F00900F550625DD8A4A2EF00F0150EB2
:100130000EEC00F05A0AD8B4D5EF01F064EC00F0F0
:1001400097EF00F08B928B9042EC00F00A0E606FFC
:100150008B8057EC00F08B9057EC00F0602FA8EFED
:1001600000F0A2EF00F0A68EF86A3F0EF76EFC0ECC
:10017000F66E000E606F400E616FED0E626FDE0E68
:10018000636F0900F550631B0900F550621B020EF6
:10019000605F000E615B60516111D8A4C1EF00F097
:1001A000621F631F62516311D8A46CEF00F0A68E2A
:1001B000F86A3F0EF76EFA0EF66E0900F550676F9B
:1001C0000900F550666FA68EF86A7F0EF76EF60E80
:1001D000F66E0900F550696F0900F550686F6651B9
:1001E000685D67516959D8A06CEF00F08B828B80F5
:1001F000F00E606F000E616FF86A040EF76E000E6D
:10020000F66EA68EA69CA688A684550EA76EAA0E8C
:10021000A76EA682400EF626D8B0F72A010E605FC0
:10022000000E615B60516011D8A401EF01F0000E77
:10023000606F3C0E616FF86A040EF76E000EF66E8A
:100240000900FF0EF55CD8A4F6EF00F0010E605F28
:10025000000E615B60516111D8A420EF01F0F00E37
:10026000616FF86A040E656F000E646F61A98B9070
:1002700061B98B8064C0F6FF65C0F7FF000EF626FB
:10028000400EF72200EE6BF0400E606F0900F5CFD4
:10029000EEFF602F46EF01F064C0F6FF65C0F7FF88
:1002A00000EE6BF0400E606FEECFF5FF0D00602F9B
:1002B00054EF01F064C0F6FF65C0F7FFA68EA69C60
:1002C000A698A684550EA76EAA0EA76EA682400E0B
:1002D0006427D8B0652B612F36EF01F08B928B909D
:1002E00064EC00F0000E806E400E816E400E826E57
:1002F0003E0E926E820E936EA00E946E2C0EE8CF80
:1003000038FF000EE8CF39FF200EE8CF3AFF000E8D
:10031000E8CFC1FF3E0EE8CFC0FF000EE8CF79FF67
:10032000E8CF78FFE8CF77FFF19E0001A2EF03F05E
:10033000150E0EEC00F05A0AD8A4B3EF00F0A68E0A
:10034000F86A000EF76E000EF66EFE0E606F3F0E3E
:10035000616FED0E626FDE0E636F0900F550631B77
:100360000900F550621B020E605F000E615B605178
:100370006111D8A4ADEF01F0621F631F0900F550B1
:10038000635DD8A4B3EF00F00900F550625DD8A416
:10039000B3EF00F0150E0EEC00F05A0AD8B4D5EF0A
:1003A00001F064EC00F0CAEF01F0A2EF03F0FFFFF0
:1003B000FFFFFFFFFFFFFFFFFFFFFFFFFFFFFFFF4D
:1003C000FFFFFFFFFFFFFFFFFFFFFFFFFFFFFFFF3D
:1003D000FFFFFFFFFFFFFFFFFFFFFFFFFFFFFFFF2D
:1003E000FFFFFFFFFFFFFFFFFFFFFFFFFFFFFFFF1D
:1003F000FFFFFFFFFFFFFFFFFFFFFFFFFFFFFFFF0D
:100400004154000041544530000041542B434C54AA
:10041000533D3100000041542657000041542B4306
:10042000434C4B3F000041542B434D47463D310068
:10043000000041542B435245473F000041542B4399
:100440004D47533D220000002B32373832353130D2
:10045000353738322200000043656E7465722050D3
:1004600069766F74204F4132392000002C206D6F67
:1004700064653D4155544F4D4154494300002C2083
:100480006D6F64653D4D414E55414C0000002C2080
:100490006661756C742072656C61793D454E4142B0
:1004A0004C45440000002C206661756C7420726518
:1004B0006C61793D44495341424C454400004154EC
:1004C0002B434D474C3D22414C4C220000004154EF
:1004D0002B434D47533D000041542B434D47443D72
:1004E000000041542B435351000041542B43494DCC
:1004F0004900000041542B43474154543F00000041
:1005000041542B53415042523D332C312C22434F06
:100510004E54595045222C2247505253220000007D
:1005200041542B53415042523D332C312C224150E7
:100530004E222C22494E5445524E45542200000072
:1005400041542B53415042523D312C310000415413
:100550002B53415042523D322C31000041542B4824
:10056000545450494E495400000041542B485454AF
:1005700050504152413D22434944222C3100000059
:1005800041542B48545450504152413D2255524CF5
:10059000222C22687474703A2F2F6661726D696E16
:1005A000672E6167726967656C2E636F2E7A612FA3
:1005B000696E6465782F6170692F6170695F64612D
:1005C00074612E7068702200000041542B4854540E
:1005D00050504152413D22434F4E54454E54222CDF
:1005E000226170706C69636174696F6E2F782D770A
:1005F00077772D666F726D2D75726C656E636F64A3
:1006000065642200000041542B4854545044415426
:10061000413D00002C313030303000006E616D659E
:100620003D616A61785F70696E6700006E616D653B
:100630003D726426646174613D33413831000000CD
:100640003044000041542B48545450414354494FC6
:100650004E3D3100000041542B4854545052454106
:100660004400000041542B485454505445524D000E
:10067000000041542B53415042523D302C31000078
:100680004F4B00004154000041544530000045529A
:10069000524F520000002B435245473A20302C3134
:1006A00000002B435245473A20302C35000041547E
:1006B0002B4350494E3F00002B4350494E3A2052A5
:1006C0004541445900002B4350494E3A2053494D6F
:1006D0002050494E00002B435343413A00002B4326
:1006E0004D47533A00002B434D474C3A00002B43F3
:1006F000474154543A20310000002B53415042529C
:100700003A000000444F574E4C4F414400002B48E4
:10071000545450414354494F4E3A00002B485454CE
:1007200050524541443A00002B48545450544552CD
:100730004D0000002B43434C4B3A00002B435351D8
:100740003A000000ABEF05F00A0A0A0A0A0A0A0A90
:100750000A0A0D4167726967656C20466C6F7720E5
:10076000436F6E74726F6C2056616C76652000006A
:100770000A0A0D3F203D20436F6D6D616E64204875
:10078000656C700A0A0D000061203D204175746F90
:100790006D617469630A0D00000063203D20436CA5
:1007A0006F73652076616C76652031207374657097
:1007B0002C20284F4E4C5920494E204D414E55413A
:1007C0004C290A0D000043203D20436C6F736520C7
:1007D00076616C7665203130302073746570732CCF
:1007E00020284F4E4C5920494E204D414E55414CEA
:1007F000290A0D00000064203D2044656372656D88
:10080000656E742076616C7665206E756D626572BA
:100810000A0D000066203D20466C6F77206D6574E0
:10082000657220646174610A0D00000069203D203A
:10083000496E6372656D656E742076616C766520B5
:100840006E756D6265720A0D00006B203D204B6174
:100850006C6962726174696F6E0A0D0000006D2030
:100860003D204D616E75616C0A0D00006F203D20CA
:100870004F70656E2076616C7665203120737465EB
:10088000702C20284F4E4C5920494E204D41425546
:10089000414C290A0D0000004F203D204F70656E2D
:1008A0002076616C7665203130302073746570730A
:1008B0002C20284F4E4C5920494E204D414E554139
:1008C0004C290A0D000070203D205061636B657457
:1008D00020646174610A0D00000072203D205265A1
:1008E00073657420666C6F772070756C7365206318
:1008F0006F756E7465720A0D000076203D2056619A
:100900006C766520646174610A0D0A0D0000356D16
:1009100073202020454550202020434F4D0A0D00D4
:100920000000356D732020202050562020202020EC
:100930002053502020202020204E455720202020CA
:100940002055464F320A0D000000436F756E740A41
:100950000D0000002020202020202020202020200A
:1009600020202020000043656E7465725069766F08
:1009700074466C6F77200000436F6E74726F6C6CFE
:100980006572204F4132392000004155544F2047B5
:100990005541524445442020202000004155544FE9
:1009A00020212143415554494F4E21210000202050
:1009B0002020202020202020202020202020000077
:1009C0004D414E55414C204755415244454420200D
:1009D00000004D414E55414C202143415554494F53
:1009E0004E21000020202020202020202020202018
:1009F000202020200000202020456469743F204EE4
:100A00006F20202020200000202020456469743FB2
:100A10002059657320202020000053657474696E8E
:100A20006773204D656E753A202000005365742071
:100A3000706F696E743A20000000466C6F77207307
:100A4000657420706F696E743A200000466C6F7791
:100A500020726174652069733A202020000053657C
:100A60006C656374204D4F44453A202020200000DF
:100A700020202020204D414E55414C202020202078
:100A8000000020202020204155544F4D415449431F
:100A9000202000004641554C542072656C61793A23
:100AA0002020202000002020202020454E41424CC4
:100AB00045202020202000002020202020444953D1
:100AC00041424C45202020200000534D53207069A6
:100AD0006E2E2E2E3A200000534D532070696E3A30
:100AE00020202020202020200000534D5320616C26
:100AF000657274733A2020202020000020202020DE
:100B000020454E41424C452020202020000020203E
:100B100020202044495341424C4520202020000001
:100B2000416C657274206D756D6265723A2020208B
:100B30000000212120464C4F57204641554C54205F
:100B400021210000504F57455220444F574E202F2F
:100B500020534554000001011F0EAF6E010EB06E10
:100B6000080EB86E260EAC6E900EAB6E230E756E30
:100B7000000E766E080E706E220E726E980E716EFA
:100B8000CF68CE68810ECD6E6C0EBB6EBC6A3E0E19
:100B9000BA6E330EB16E000EB46E4E6AB36AB26AAC
:100BA000010E6E6F6F6B706B020E716F726B736BF9
:100BB000030E746F756B766B040E776F786B796BC1
:100BC000050E7A6F7B6B7C6B060E7D6F7E6B7F6B89
:100BD000070E806F816B826B080E836F846B856B51
:100BE000090E866F876B886B0A0E896F8A6B8B6B19
:100BF000F26A9F6AA26AA56AF08CF08E9F80A28238
:100C0000F19AF1989D8AA38A9D809D82A192A082EB
:100C1000F086F088006A016A026A036A046A056A5B
:100C2000066A076A086A346B356B080E186E640E24
:100C3000366FC80E376FAE6B028C0A0E4B6E4C6A65
:100C4000000E4D6E000E5F6FB16BB26BF90E386F18
:100C5000396F3E0E3A6F3B6F7F0E3C6F3D6FFF0E5C
:100C60003E6F3F6FB2CF4CF1B3CF4DF14EC04EF15E
:100C7000A56BA66BA76BB2CF55F1B3CF56F14EC0A3
:100C800057F1AA6BAB6BAC6B020E5D6F020E5E6F21
:100C90003C0E476E000E486ED00E496E070E4A6E2F
:100CA000100E996F270E9A6F000E9B6FA16FA26FA7
:100CB000000E516E000E536E000E506E000E526EFE
:100CC000000EBC6FFF0EB56F000E0EEC00F0996FBA
:100CD000010E0EEC00F09A6F020E0EEC00F0076EA3
:100CE000030E0EEC00F0EA6F040E0EEC00F0EB6F5A
:100CF000050E0EEC00F0EC6F060E0EEC00F0ED6F42
:100D0000080E0EEC00F0E8CFABF0090E0EEC00F090
:100D1000E8CFACF00A0E0EEC00F0E8CFADF00B0E11
:100D20000EEC00F0E8CFAEF00C0E0EEC00F0E8CFC9
:100D3000AFF00D0E0EEC00F0E8CFB0F00E0E0EECA2
:100D400000F0E8CFB1F00F0E0EEC00F0E8CFB2F0FB
:100D5000100E0EEC00F0E8CFB3F0110E0EEC00F028
:100D6000E8CFB4F01EEC32F0C80E9C5DD8A0BBEF0B
:100D700006F0640E9C6FE80E9D6F9F6F030E9E6FD2
:100D8000A06FD890A0339F33D890A0339F33676B68
:100D90008286949694880000000000000000000005
:100DA0000000000000000000000000000000080E2D
:100DB000186E000E196E18EC1BF01950AEEC1BF0FB
:100DC0009EEC26F04CEC00F018EC1BF01950AEEC49
:100DD0001BF0300E196E0EEC1CF0B4EC12F00EECA1
:100DE0001CF0B4EC12F00EEC1CF0B4EC12F0200E7F
:100DF000196E0EEC1CF0B4EC12F0280EC3EC22F0CD
:100E0000B4EC12F0080EC3EC22F0B4EC12F0010EB8
:100E1000C3EC22F0B4EC12F0B4EC12F00C0EC3EC04
:100E200022F0B4EC12F0800EC3EC22F0B4EC12F01D
:100E3000090E186E126B040E176F8A0E1E6F290EA4
:100E40001F6F81A2179781B21787A86B81A4129395
:100E500081B41283AD6BFF0EB66F420E126E8A8A9A
:100E6000276A286AC80EB86F000EB96F606B616B95
:100E70001E0E5F6ED08EF28EF28C020EE86F040EA4
:100E8000E96FA68EF86A070EF76E480EF66EF5EC5F
:100E900026F055EC27F0A68EF86A070EF76E700E56
:100EA000F66EF5EC26F05250D8A45BEF07F0ABECF1
:100EB00010F00DEC0EF0E1EC11F069EC27F066ECAF
:100EC00007F006804FEC2BF053EF07F05250D8B4E8
:100ED00082EF07F004BA78EF07F004B878EF07F074
:100EE00004B078EF07F004B278EF07F07CEF07F07A
:100EF000700E5D6E170E5E6E5D505E10D8A482EFB0
:100F000007F0FF00FB6A0F0EFA6E5250E834E83427
:100F1000FC0B1A0FD8B0FA2AF96E13EF08F023EF82
:100F200008F044EF08F066EF08F087EF08F0B0EF44
:100F300008F0D2EF08F0F3EF08F01CEF09F058EFDB
:100F400009F094EF09F0D0EF09F00EEF0AF03CEF52
:100F50000AF051EF0AF054EF0AF082EF0AF097EF2F
:100F60000AF09AEF0AF0C7EF0AF0E9EF0AF00AEF89
:100F70000BF03CEF0BF076EF0BF0B0EF0BF0EAEF7D
:100F80000BF020EF0CF00FEF08F00FEF08F00FEF71
:100F900008F00FEF08F00FEF08F00FEF08F00FEF79
:100FA00008F00FEF08F00FEF08F00FEF08F00FEF69
:100FB00008F00FEF08F00FEF08F00FEF08F00FEF59
:100FC00008F00FEF08F00FEF08F00FEF08F00FEF49
:100FD00008F00FEF08F00FEF08F00FEF08F00FEF39
:100FE00008F00FEF08F00FEF08F00FEF08F00FEF29
:100FF00008F00FEF08F00FEF08F00FEF08F00FEF19
:1010000008F00FEF08F00FEF08F00FEF08F00FEF08
:1010100008F00FEF08F00FEF08F00FEF08F0000EE8
:10102000526E31EF0DF004A218EF08F0049207722F
:1010300004AA21EF08F0049A522A700E5D6E170E72
:101040005E6E31EF0DF0A68EF86A0A0EF76E1A0E7C
:10105000F66E03EC27F0A68EF86A0A0EF76E080EFD
:10106000F66E12EC27F0C90EC3EC22F0B4EC12F0CD
:101070000F0EC3EC22F0B4EC12F00492049804902A
:10108000049A522A31EF0DF004A24CEF08F00492BA
:10109000522A522A64EF08F004B852EF08F004A074
:1010A00064EF08F004980490A68EF86A090EF76EB3
:1010B000F60EF66E12EC27F0C90EC3EC22F0B4EC7B
:1010C00012F0522AD0EF08F031EF0DF004A26DEFCC
:1010D00008F00492526A85EF08F004B873EF08F044
:1010E00004A085EF08F004980490A68EF86A0A0E12
:1010F000F76E080EF66E12EC27F0C90EC3EC22F064
:10110000B4EC12F05206D0EF08F031EF0DF0A68EDD
:10111000F86A0A0EF76E2C0EF66E03EC27F08B0EB3
:10112000B76F99512B6E9A512C6E21EC27F0A68E39
:10113000F86A090EF76EF60EF66E12EC27F0C90E7D
:10114000C3EC22F0B4EC12F00F0EC3EC22F0B4ECBE
:1011500012F0049204980490049A522A31EF0DF090
:1011600004A2B8EF08F00492070E5226D0EF08F060
:1011700004B8BEEF08F004A0D0EF08F00498049083
:10118000A68EF86A0A0EF76E080EF66E12EC27F0BD
:10119000C90EC3EC22F0B4EC12F0522AD0EF08F0E2
:1011A00031EF0DF004A2D9EF08F00492522AF1EFCA
:1011B00008F004B8DFEF08F004A0F1EF08F004989D
:1011C0000490A68EF86A090EF76EF60EF66E12EC13
:1011D00027F0C90EC3EC22F0B4EC12F05206F1EF86
:1011E00008F031EF0DF0A68EF86A0A0EF76E3A0E8F
:1011F000F66E03EC27F0A68EF86A090EF76E540E11
:10120000F66E12EC27F0C60EB76F99512B6E9A51FD
:101210002C6E3DEC27F0C90EC3EC22F0B4EC12F0BA
:101220000F0EC3EC22F0B4EC12F004920498049078
:10123000049A522A31EF0DF004A834EF09F0049813
:101240002E2A0A0E2E5C000ED8B02E6EC90EC3ECEC
:1012500022F0B4EC12F02E50300FCAEC22F0C90E7E
:10126000C3EC22F0B4EC12F004A04CEF09F00490AF
:101270002E060A0E2E5C090ED8B02E6EC90EC3ECD7
:1012800022F0B4EC12F02E50300FCAEC22F0C90E4E
:10129000C3EC22F0B4EC12F004A256EF09F0049271
:1012A000C80EC3EC22F0B4EC12F0522A31EF0DF06C
:1012B00004A870EF09F004982F2A0A0E2F5C000E84
:1012C000D8B02F6EC80EC3EC22F0B4EC12F02F5041
:1012D000300FCAEC22F0C80EC3EC22F0B4EC12F0CE
:1012E00004A088EF09F004902F060A0E2F5C090E67
:1012F000D8B02F6EC80EC3EC22F0B4EC12F02F5011
:10130000300FCAEC22F0C80EC3EC22F0B4EC12F09D
:1013100004A292EF09F00492C70EC3EC22F0B4ECE1
:1013200012F0522A31EF0DF004A8ACEF09F0049846
:10133000302A0A0E305C000ED8B0306EC70EC3ECF7
:1013400022F0B4EC12F03050300FCAEC22F0C70E8D
:10135000C3EC22F0B4EC12F004A0C4EF09F0049046
:1013600030060A0E305C090ED8B0306EC70EC3ECE2
:1013700022F0B4EC12F03050300FCAEC22F0C70E5D
:10138000C3EC22F0B4EC12F004A2CEEF09F0049208
:10139000C60EC3EC22F0B4EC12F0522A31EF0DF07D
:1013A00004A8E8EF09F00498312A020E315C000E1F
:1013B000D8B0316EC60EC3EC22F0B4EC12F031504E
:1013C000300FCAEC22F0C60EC3EC22F0B4EC12F0DF
:1013D00004A000EF0AF004903106020E315C010E09
:1013E000D8B0316EC60EC3EC22F0B4EC12F031501E
:1013F000300FCAEC22F0C60EC3EC22F0B4EC12F0AF
:1014000004A20CEF0AF00492FBEC16F02B50996F3B
:101410002C509A6F070E525E31EF0DF0A68EF86ACF
:101420000A0EF76E5E0EF66E03EC27F007A023EFB0
:101430000AF0A68EF86A0A0EF76E700EF66E12ECBF
:1014400027F02BEF0AF0A68EF86A0A0EF76E820ECE
:10145000F66E12EC27F0C50EC3EC22F0B4EC12F0DD
:101460000F0EC3EC22F0B4EC12F004920498049036
:10147000049A522A31EF0DF004B842EF0AF004A0AA
:1014800048EF0AF004980490077052064FEF0AF0F4
:1014900004A24FEF0AF00492522A4FEF0AF031EF04
:1014A0000DF0522A31EF0DF0A68EF86A0A0EF76E93
:1014B000940EF66E03EC27F007A269EF0AF0A68EF1
:1014C000F86A0A0EF76EA60EF66E12EC27F071EFB0
:1014D0000AF0A68EF86A0A0EF76EB80EF66E12ECD7
:1014E00027F0C50EC3EC22F0B4EC12F00F0EC3ECE3
:1014F00022F0B4EC12F0049204980490049A522A58
:1015000031EF0DF004B888EF0AF004A08EEF0AF076
:10151000049804900772520695EF0AF004A295EF22
:101520000AF00492522A95EF0AF031EF0DF0522A98
:1015300031EF0DF0A68EF86A0A0EF76ECA0EF66E3F
:1015400003EC27F0EA51CAEC22F0EB51CAEC22F08E
:10155000EC51CAEC22F0ED51CAEC22F0A68EF86AEA
:10156000090EF76EF60EF66E12EC27F0C90EC3ECFC
:1015700022F0B4EC12F00F0EC3EC22F0B4EC12F037
:10158000049204980490049A522A31EF0DF004A2B8
:10159000CFEF0AF00492070E5226E7EF0AF004B8E4
:1015A000D5EF0AF004A0E7EF0AF004980490A68EA5
:1015B000F86A0A0EF76E080EF66E12EC27F0C90EE6
:1015C000C3EC22F0B4EC12F0522AE7EF0AF031EF4C
:1015D0000DF004A2F0EF0AF00492522A08EF0BF08B
:1015E00004B8F6EF0AF004A008EF0BF0049804909A
:1015F000A68EF86A090EF76EF60EF66E12EC27F05C
:10160000C90EC3EC22F0B4EC12F0520608EF0BF056
:1016100031EF0DF0A68EF86A0A0EF76ED80EF66E50
:1016200003EC27F0A68EF86A090EF76E540EF66EDC
:1016300012EC27F0C60EC3EC22F0B4EC12F0EA5123
:10164000CAEC22F0EB51CAEC22F0EC51CAEC22F0C9
:10165000ED51CAEC22F0C90EC3EC22F0B4EC12F04A
:101660000F0EC3EC22F0B4EC12F004920498049034
:10167000049A522A31EF0DF004A853EF0BF00498AE
:10168000ED2B3A0EED5D300ED8B0ED6FC90EC3EC08
:1016900022F0B4EC12F0ED51CAEC22F0C90EC3EC0A
:1016A00022F0B4EC12F004A06AEF0BF00490ED0706
:1016B000300EED5D390ED8A0ED6FC90EC3EC22F0EF
:1016C000B4EC12F0ED51CAEC22F0C90EC3EC22F0DA
:1016D000B4EC12F004A274EF0BF00492C80EC3EC49
:1016E00022F0B4EC12F0522A31EF0DF004A88DEF85
:1016F0000BF00498EC2B3A0EEC5D300ED8B0EC6F8A
:10170000C80EC3EC22F0B4EC12F0EC51CAEC22F09B
:10171000C80EC3EC22F0B4EC12F004A0A4EF0BF05E
:101720000490EC07300EEC5D390ED8A0EC6FC80EBB
:10173000C3EC22F0B4EC12F0EC51CAEC22F0C80E6B
:10174000C3EC22F0B4EC12F004A2AEEF0BF0049262
:10175000C70EC3EC22F0B4EC12F0522A31EF0DF0B8
:1017600004A8C7EF0BF00498EB2B3A0EEB5D300E9C
:10177000D8B0EB6FC70EC3EC22F0B4EC12F0EB5113
:10178000CAEC22F0C70EC3EC22F0B4EC12F004A0B5
:10179000DEEF0BF00490EB07300EEB5D390ED8A0B6
:1017A000EB6FC70EC3EC22F0B4EC12F0EB51CAECB5
:1017B00022F0C70EC3EC22F0B4EC12F004A2E8EF62
:1017C0000BF00492C60EC3EC22F0B4EC12F0522AD5
:1017D00031EF0DF004A801EF0CF00498EA2B3A0E5B
:1017E000EA5D300ED8B0EA6FC60EC3EC22F0B4EC5E
:1017F00012F0EA51CAEC22F0C60EC3EC22F0B4ECAF
:1018000012F004A018EF0CF00490EA07300EEA5D25
:10181000390ED8A0EA6FC60EC3EC22F0B4EC12F079
:10182000EA51CAEC22F0C60EC3EC22F0B4EC12F07E
:1018300004A21EEF0CF00492070E525E31EF0DF081
:10184000000E0EEC00F0995DD8B42EEF0CF099511B
:1018500014EC00F0ABEC12F020EF0CF0010E0EECEB
:1018600000F09A5DD8B43CEF0CF09A5114EC00F003
:10187000ABEC12F02EEF0CF0020E0EEC00F0075C59
:10188000D8B44AEF0CF0075014EC00F0ABEC12F0B7
:101890003CEF0CF0030E0EEC00F0EA5DD8B458EF0C
:1018A0000CF0EA5114EC00F0ABEC12F04AEF0CF043
:1018B000040E0EEC00F0EB5DD8B466EF0CF0EB51CB
:1018C00014EC00F0ABEC12F058EF0CF0050E0EEC3F
:1018D00000F0EC5DD8B474EF0CF0EC5114EC00F0B7
:1018E000ABEC12F066EF0CF0060E0EEC00F0ED5DC6
:1018F000D8B482EF0CF0ED5114EC00F0ABEC12F028
:1019000074EF0CF0080E0EEC00F0ABC0E8FFA85C22
:10191000D8B493EF0CF0ABC0E8FF14EC00F0ABECE4
:1019200012F082EF0CF0090E0EEC00F0ACC0E8FFF4
:10193000A85CD8B4A4EF0CF0ACC0E8FF14EC00F045
:10194000ABEC12F093EF0CF00A0E0EEC00F0ADC011
:10195000E8FFA85CD8B4B5EF0CF0ADC0E8FF14EC1C
:1019600000F0ABEC12F0A4EF0CF00B0E0EEC00F05C
:10197000AEC0E8FFA85CD8B4C6EF0CF0AEC0E8FF7C
:1019800014EC00F0ABEC12F0B5EF0CF00C0E0EEC1A
:1019900000F0AFC0E8FFA85CD8B4D7EF0CF0AFC040
:1019A000E8FF14EC00F0ABEC12F0C6EF0CF00D0EFB
:1019B0000EEC00F0B0C0E8FFA85CD8B4E8EF0CF083
:1019C000B0C0E8FF14EC00F0ABEC12F0D7EF0CF075
:1019D0000E0E0EEC00F0B1C0E8FFA85CD8B4F9EF31
:1019E0000CF0B1C0E8FF14EC00F0ABEC12F0E8EF43
:1019F0000CF00F0E0EEC00F0B2C0E8FFA85CD8B4FB
:101A00000AEF0DF0B2C0E8FF14EC00F0ABEC12F0FE
:101A1000F9EF0CF0100E0EEC00F0B3C0E8FFA85C7C
:101A2000D8B41BEF0DF0B3C0E8FF14EC00F0ABEC42
:101A300012F00AEF0DF0110E0EEC00F0B4C0E8FF4A
:101A4000A85CD8B42CEF0DF0B4C0E8FF14EC00F0A3
:101A5000ABEC12F01BEF0DF0040E506E526A31EF3A
:101A60000DF012001200000E386E000E396E280EB6
:101A70003A6E010E3B6E000E3C6EA5C13DF0A6C154
:101A80003EF0A7C13FF0406A416A41EC18F0090EF0
:101A90008C6F01EE6EF0EE2E5BEF0DF0ED50E9CFA6
:101AA00090F1EACF91F1090EEE6E38C0EEFF39C029
:101AB000EEFF5DEF0DF0EE50EE508C2F4BEF0DF082
:101AC00090C1E9FF91C1EAFF6E0EE95CD8A46EEF08
:101AD0000DF0010EEA58D8B490EF0DF0860EE95CD7
:101AE000D8A478EF0DF0010EEA58D8B4C7EF0DF086
:101AF000EE50EE50EE50EE503850EE5C3950EE584D
:101B0000D8A090EF0DF0080EE95E000EEA5AEE50F4
:101B1000385CEE503958D8A0C7EF0DF0FCEF0DF04F
:101B200090C1E9FF91C1EAFF90C1E1FF91C1E2FFDD
:101B3000860EE95CD8A4A2EF0DF0010EEA58D8B4E5
:101B4000C5EF0DF0EE50EE50EE50EE503850EE5C1A
:101B50003950EF58D8B0C5EF0DF0EDCF8FF1EDCF84
:101B60008EF1EFCF8DF1E6CFEEFFE6CFEEFFE7CFC0
:101B7000EFFF8FC1E5FF8EC1E5FF8DC1E6FFE650A7
:101B8000E650ED50ED5098EF0DF0FCEF0DF090C1E8
:101B9000E9FF91C1EAFF90C1E1FF91C1E2FF6E0E42
:101BA000E95CD8A4D9EF0DF0010EEA58D8B4FAEFE9
:101BB0000DF0ED50ED50EE50385CEF503958D8B084
:101BC000FAEF0DF0EDCF8FF1EDCF8EF1EFCF8DF17C
:101BD000E6CFEEFFE6CFEEFFE7CFEFFF8FC1E5FFE9
:101BE0008EC1E5FF8DC1E5FFE550E550ED50ED50AC
:101BF000CFEF0DF0FCEF0DF07BC138F07CC139F078
:101C00003A6A3B6A3C6A38C0A1F139C0A2F1A151DD
:101C1000F227A251F323F42B1200FB6A1C0EFA6E7A
:101C20005050E834E8347C0B300FD8B0FA2AF96E03
:101C30005CEF0EF060EF0EF078EF0EF081EF0EF03B
:101C400095EF0EF0B2EF0EF0D8EF0FF0DCEF0FF0E3
:101C500001EF10F082EF10F086EF10F058EF0EF069
:101C600058EF0EF058EF0EF058EF0EF058EF0EF060
:101C700058EF0EF058EF0EF058EF0EF058EF0EF050
:101C800058EF0EF058EF0EF058EF0EF058EF0EF040
:101C900058EF0EF058EF0EF058EF0EF058EF0EF030
:101CA00058EF0EF058EF0EF058EF0EF058EF0EF020
:101CB000000E506E0DEF0EF0010E506E9BEF10F007
:101CC000A68EF86A090EF76E660EF66E03EC27F024
:101CD000A68EF86A090EF76E780EF66E12EC27F0F3
:101CE000FA0E106E000E116E020E506E9BEF10F089
:101CF00010501110D8A47FEF0EF0030E506E9BEF22
:101D000010F0A68EF86A090EF76E540EF66E03EC0C
:101D100027F0A68EF86A090EF76E540EF66E12ECD6
:101D200027F0040E506E9BEF10F007A29AEF0EF012
:101D3000A4EF0EF0A68EF86A090EF76E9C0EF66EF2
:101D400003EC27F0AEEF0EF0A68EF86A090EF76EE0
:101D50008A0EF66E03EC27F0AEEF0EF0050E506E15
:101D600028EF00F007B0BAEF0EF060516111D8B45F
:101D7000BEEF0EF0060E506ED6EF0FF005AAD6EFAE
:101D80000FF0059A8A7407A2C8EF0EF0D2EF0EF09A
:101D9000A68EF86A090EF76E9C0EF66E03EC27F01D
:101DA000DCEF0EF0A68EF86A090EF76E8A0EF66E5C
:101DB00003EC27F0DCEF0EF0C20EB76FF451D8A49D
:101DC000E8EF0EF0A1512B6EA2512C6EFFEF0EF03A
:101DD000F2C138F0F3C139F03A6A3B6A3C6AF4C1A7
:101DE0003DF03E6A3F6A406A416A41EC18F038C0F3
:101DF0002BF039C02CF038C0F5F139C0F6F1F26B98
:101E0000F36BF46B49EC29F021EC27F09CEC10F01B
:101E1000CAEC22F0C80EB76F99512B6E9A512C6EF6
:101E200021EC27F0D6EF0FF09BB1BAEF0EF08A88C5
:101E3000B80E276E0B0E286E506ED6EF0FF0F29E86
:101E400047504810F28ED8B459EC12F003ACD6EFDC
:101E50000FF0039CF29E9951A15D5A6F9A51A259BD
:101E60005B6FF28ED8A037EF0FF03CEF0FF08AB81F
:101E7000986B8A9841EF0FF08AA8986B8A8841EF97
:101E80000FF05A515B11D8B4D5EF0FF0D8B04FEF27
:101E90000FF05A1F5B1F010E5A27000E5B23F40E32
:101EA0005A5D010E5B59D8A05EEF0FF0982B190E0A
:101EB000985D190ED8B0986F5FEF0FF0986B880E91
:101EC0005A5D130E5B59D8A06CEF0FF0800E5A6F5D
:101ED000000E5B6FC0EF0FF0600E5A5D090E5B598C
:101EE000D8A079EF0FF0400E5A6F000E5B6FC0EF75
:101EF0000FF0400E5A5D060E5B59D8A086EF0FF02A
:101F0000200E5A6F000E5B6FC0EF0FF0900E5A5DFF
:101F1000010E5B59D8A093EF0FF0100E5A6F000E10
:101F20005B6FC0EF0FF0C80E5A5D000E5B59D8A072
:101F3000A0EF0FF0080E5A6F000E5B6FC0EF0FF0AE
:101F4000640E5A5D000E5B59D8A0ADEF0FF0040E81
:101F50005A6F000E5B6FC0EF0FF00A0E5A5D000E55
:101F60005B59D8A0BAEF0FF0020E5A6F000E5B6FEC
:101F7000C0EF0FF0000E5A6F000E5B6FC0EF0FF056
:101F80005A51275C5B512858D8B0D6EF0FF05AC190
:101F900027F05BC128F027502810D8B4272A985181
:101FA0002726000E2822D6EF0FF0986B9BEF10F03B
:101FB000070E506E9BEF10F007A2E1EF0FF0EBEF72
:101FC0000FF0A68EF86A090EF76ED20EF66E03ECCD
:101FD00027F0F5EF0FF0A68EF86A090EF76EC00E27
:101FE000F66E03EC27F0F5EF0FF0A68EF86A090EF7
:101FF000F76EE40EF66E12EC27F0080E506E28EF26
:1020000000F007B00DEF10F060516111D8A40DEF92
:1020100010F0090E506E80EF10F005AA80EF10F05E
:10202000059A07B02FEF10F0870EC3EC22F0B4EC46
:1020300012F0200ECAEC22F0200ECAEC22F0200E84
:10204000CAEC22F0200ECAEC22F08B0EB76F605162
:102050002B6E61512C6E21EC27F04AEF10F007A295
:1020600034EF10F03EEF10F0A68EF86A090EF76E0E
:10207000D20EF66E03EC27F048EF10F0A68EF86A49
:10208000090EF76EC00EF66E03EC27F048EF10F065
:102090004AEF10F0C20EB76FF451D8A456EF10F00B
:1020A000A1512B6EA2512C6E6DEF10F0F2C138F0E1
:1020B000F3C139F03A6A3B6A3C6AF4C13DF03E6ACA
:1020C0003F6A406A416A41EC18F038C02BF039C0D1
:1020D0002CF038C0F5F139C0F6F1F26BF36BF46B0C
:1020E00021EC27F09CEC10F0CAEC22F0C80EB76F80
:1020F00099512B6E9A512C6E21EC27F080EF10F045
:102100009BEF10F0040E506E9BEF10F0A68EF86A55
:102110000B0EF76E320EF66E03EC27F0A68EF86A01
:102120000B0EF76E440EF66E12EC27F0818004B2AF
:10213000FF009BEF10F01200FB6A210EFA6E535065
:10214000532AE834060B4E0FD8B0FA2AF96E2F0C3A
:102150002D0CCD0C7C0C190E04A8AF6F04A8C6EF93
:1021600010F0190EB06FAE51D8A4C6EF10F00F0EDC
:10217000AE6F900E606F010E616F8A98140EAF27DC
:10218000FF0ED8B0AF6FAF51276E286A190E04A0AA
:10219000B06F04A0E1EF10F0190EAF6FAE51D8A4EC
:1021A000E1EF10F00F0EAE6F900E606F010E616FD9
:1021B0008A88140EB027FF0ED8B0B06FB051276ECA
:1021C000286A12009DEC29F0D8A0DFEF11F08B7087
:1021D0003F0AD8B426EF11F05E0AD8B4AFEF11F081
:1021E000200AD8B4AFEF11F0220AD8B4B3EF11F03F
:1021F000200AD8B4B9EF11F0250AD8B4BFEF11F016
:10220000200AD8B4BFEF11F02D0AD8B4C5EF11F0F1
:10221000200AD8B4C5EF11F0260AD8B4C9EF11F0DE
:10222000200AD8B4C9EF11F0220AD8B4CDEF11F0CA
:10223000200AD8B4D3EF11F0390AD8B4D9EF11F08D
:10224000200AD8B4D9EF11F0DFEF11F0A68EF86AAA
:10225000070EF76E480EF66EF5EC26F055EC27F0FB
:10226000A68EF86A070EF76E700EF66EF5EC26F085
:10227000A68EF86A070EF76E880EF66EF5EC26F05D
:10228000A68EF86A070EF76E9A0EF66EF5EC26F03B
:10229000A68EF86A070EF76EC60EF66EF5EC26F0FF
:1022A000A68EF86A070EF76EF60EF66EF5EC26F0BF
:1022B000A68EF86A080EF76E140EF66EF5EC26F090
:1022C000A68EF86A080EF76E2C0EF66EF5EC26F068
:1022D000A68EF86A080EF76E4A0EF66EF5EC26F03A
:1022E000A68EF86A080EF76E5E0EF66EF5EC26F016
:1022F000A68EF86A080EF76E6C0EF66EF5EC26F0F8
:10230000A68EF86A080EF76E980EF66EF5EC26F0BB
:10231000A68EF86A080EF76EC60EF66EF5EC26F07D
:10232000A68EF86A080EF76EDA0EF66EF5EC26F059
:10233000A68EF86A070EF76EF60EF66EF5EC26F02E
:10234000A68EF86A080EF76EFA0EF66EF5EC26F019
:10235000C80E4B6E050E4C6E029CDFEF11F0050EA1
:10236000506EDFEF11F08A88010E276E286ADFEFCA
:1023700011F08A88640E276E286ADFEF11F0019A47
:10238000019C000E5F6FDFEF11F0030E5F6FDFEF58
:1023900011F0080E506EDFEF11F08A98010E276ED3
:1023A000286ADFEF11F08A98640E276E286ADFEF43
:1023B00011F0019A019C020E5F6FDFEF11F0120025
:1023C00012005F51020AD8A420EF12F0280E275CF9
:1023D000000E2858D8A0F0EF11F0280EF1EF11F000
:1023E0002750096E8AA820EF12F0280E0A6E0950B5
:1023F0000A5C0B6ED8B403EF12F0200E5FEC13F002
:102400000B2EFDEF11F0630E5FEC13F00950D8B402
:1024100010EF12F0200E5FEC13F0092E0AEF12F00D
:102420007C0E5FEC13F0200E5FEC13F00A2E13EF1E
:1024300012F0200E5FEC13F062EC27F020EF12F0A8
:102440002850050ED8A4C80E6D6F27502810D8B498
:1024500058EF12F0010E275E000E285A8AB833EFAB
:1024600012F042EF12F008BC58EF12F029502A1077
:10247000D8B43FEF12F0010E295E000E2A5A630E07
:102480004FEF12F008B658EF12F02AB84CEF12F0E6
:10249000010E2926000E2A226F0E4FEF12F0C6EC15
:1024A00012F08A86C6EC12F08A966D2F25EF12F094
:1024B00012008A98F29E9F51275CA0512858D8B0EC
:1024C0006AEF12F09FC127F0A0C128F03C0E476EC2
:1024D000000E486EF28E12008A98F29E9DC127F07F
:1024E0009EC128F03C0E476E000E486EF28E120020
:1024F0008DEC12F08DEC12F08DEC12F08DEC12F0F0
:102500008DEC12F08DEC12F08DEC12F08DEC12F0DF
:102510008DEC12F08DEC12F01200ABEC12F0ABEC83
:1025200012F0ABEC12F0ABEC12F0ABEC12F0ABEC47
:1025300012F0ABEC12F0ABEC12F0ABEC12F0ABEC37
:1025400012F01200C70ED56E5E0ED66EF294F2A493
:10255000B0EF12F01200C70ED56E940ED66EF29444
:10256000F2A4B0EF12F01200C70ED56E660ED66E52
:10257000F294F2A4B0EF12F01200C70ED56EF50E71
:10258000D66EF294F2A4C2EF12F01200C70ED56E0E
:10259000FD0ED66EF294F2A4CBEF12F0120022EEF2
:1025A00000F03A513B19D8B4E1EF12F03A29400A51
:1025B000D8B4400E400AD96E3A6FDF50AD6EE2EFEC
:1025C00012F09D98120025EE00F03E513F19D8B44C
:1025D000F5EF12F03E29000AD8B4000E000AD96EB9
:1025E0003E6FDF50736EF6EF12F0A398120000906A
:1025F000ABA204EF13F00080AB98ABB8FCEF12F085
:10260000AB88ABA800EF13F0ABA409EF13F0008088
:10261000AE5000B020EF13F023EE00F03929FA0A93
:10262000D8B4FA0EFA0AD96E3819D8B41EEF13F0DE
:10263000AE50DF6ED950396F20EF13F0AE500082EC
:102640001200009071A22EEF13F00080719871B803
:1026500026EF13F0718871A82AEF13F071A433EFFD
:1026600013F00080745000B04AEF13F022EE40F0F7
:102670003D29800AD8B4C00E800AD96E3C19D8B45E
:1026800048EF13F07450DF6ED9503D6F4AEF13F0EE
:10269000745000861200166E22EE00F03B29400AAC
:1026A000D8B4400E400AD96ED9503A19D8B454EF74
:1026B00013F01650DF6ED9503B6F16501200176E94
:1026C00025EE00F03F29000AD8B4000E000AD96EAA
:1026D000D9503E19D8A472EF13F005A868EF13F093
:1026E00076EF13F01750DF6ED9503F6F175012007E
:1026F0007CEF13F094EF13F0E8CF31F1D8CF32F143
:10270000E0CF33F10101A1B265EC16F0F0B078EC46
:1027100016F0F0B28AEC16F09E9031C1E8FF32C19B
:10272000D8FF33C1E0FF1000E8CF20F1D8CF21F16E
:10273000EACF23F1E9CF22F1E2CF25F1E1CF24F175
:10274000DACF27F1D9CF26F1FACF28F1FBCF29F143
:10275000F5CF2DF1F8CF2CF1F7CF2BF1F6CF2AF1F1
:10276000F3CF2EF1F4CF2FF1E0CF30F19EBAF7EC9A
:1027700012F0ABA2C5EF13F00000AB98ABB8BDEF01
:1027800013F0AB88ABA8C1EF13F0A4BA21EC13F09F
:102790009DA8CEEF13F09EB8CFEC12F0A3A8D4EF13
:1027A00013F0A4B8E3EC12F09EB2FAEC13F020C1DF
:1027B000E8FF21C1D8FF23C1EAFF22C1E9FF25C1FB
:1027C000E2FF24C1E1FF27C1DAFF26C1D9FF28C1FA
:1027D000FAFF29C1FBFF2DC1F5FF2CC1F8FF2BC16A
:1027E000F7FF2AC1F6FF2EC1F3FF2FC1F4FF30C15E
:1027F000E0FF1000028EB12BC282362F03EF14F0DF
:10280000640E366F007EAE51D8A4AE079DB80FEFB0
:1028100014F03A513B19D8B40FEF14F09D88A3B8C7
:1028200018EF14F03E513F19D8B418EF14F0A388F4
:1028300010501110D8B423EF14F0010E105E000EEA
:10284000115A7BEF14F025EF14F0BF51C011D8B42A
:1028500032EF14F0010EBF5F000EC05BBF51C0111C
:10286000D8B4348D122E38EF14F0058A420E126E51
:1028700007B049EF14F060516111D8B450EF14F073
:10288000010E605F000E615B60516111D8B450EFC2
:1028900014F000AE8B9000BE8B808B9251EF14F041
:1028A0008B905D505E10D8B45AEF14F0010E5D5E4F
:1028B000000E5E5AB851B911D8B465EF14F0010E8C
:1028C000B85F000EB95B6CEF14F0A16BA26B07A2AE
:1028D0006CEF14F00A0E506E49504A10D8B477EFDE
:1028E00014F0010E495E000E4A5A7BEF14F0000E00
:1028F0009B6F7BEF14F047504810D8B484EF14F06E
:10290000010E475E000E485A4B2EA2EF14F04C50B9
:10291000D8A49FEF14F05F51000AD8B499EF14F0D7
:10292000010AD8B499EF14F0050AD8B499EF14F05D
:10293000028C4D50D8A44D060A0EA1EF14F04C069F
:10294000C80E4B6E090EECEC26F0C4CF6AF10D0EEA
:10295000ECEC26F06A51C45CD8B0B1EF14F0C4506E
:102960006A5D6B6F050E6B5DD8B0DEEF14F0620E22
:102970006A5DD8A0C2EF14F0689D689D689D689D4F
:1029800024EF15F0460E6A5DD8A0CDEF14F06C91DF
:102990006C836C856C9724EF15F0280E6A5DD8A0C7
:1029A000D8EF14F06C816C936C956C8724EF15F064
:1029B0006C916C936C956C9724EF15F08D0E6A5D9D
:1029C000D8A0E9EF14F06C816C83689D689D01EFDD
:1029D00015F06C0E6A5DD8A0F4EF14F06C916C8366
:1029E000689D689D01EF15F0490E6A5DD8A0FFEF64
:1029F00014F06C816C93689D689D01EF15F06C91EB
:102A00006C938D0EC45CD8A00CEF15F06C856C87B0
:102A1000689D689D24EF15F06C0EC45CD8A017EF7C
:102A200015F06C856C97689D689D24EF15F0490E34
:102A3000C45CD8A022EF15F06C956C87689D689DEA
:102A400024EF15F06C956C9704A629EF15F02EEF86
:102A500015F06CA533EF15F040EF15F06CB533EFC2
:102A600015F040EF15F09451D8B445EF15F0942FC0
:102A700045EF15F004A6049204B6048245EF15F064
:102A8000010E946F047645EF15F004A44AEF15F09B
:102A90004FEF15F06CA754EF15F061EF15F06CB720
:102AA00054EF15F061EF15F09551D8B466EF15F0BD
:102AB000952F66EF15F004A4049004B4048066EF2B
:102AC00015F0010E956F047466EF15F004AE6BEF10
:102AD00015F070EF15F06CA175EF15F082EF15F0A1
:102AE0006CB175EF15F082EF15F09651D8B487EF01
:102AF00015F0962F87EF15F004AE049A04BE048AF1
:102B000087EF15F0010E966F047E87EF15F004AC89
:102B10008CEF15F091EF15F06CA396EF15F0A3EF85
:102B200015F06CB396EF15F0A3EF15F09751D8B4EC
:102B3000A8EF15F0972FA8EF15F004AC049804BC8B
:102B40000488A8EF15F0010E976F047CA8EF15F02C
:102B500005A2ADEF15F0B2EF15F081A2B7EF15F0B9
:102B6000C4EF15F081B2B7EF15F0C4EF15F0A8511E
:102B7000D8B4C9EF15F0A82FC9EF15F005A2179723
:102B800005B21787C9EF15F00A0EA86F0572C9EFD5
:102B900015F005A4CEEF15F0D3EF15F081A4D8EF12
:102BA00015F0E5EF15F081B4D8EF15F0E5EF15F06D
:102BB000AD51D8B4EAEF15F0AD2FEAEF15F005A44A
:102BC000129305B41283EAEF15F00A0EAD6F057487
:102BD000EAEF15F0450EECEC26F0C4CF69F18E0E4D
:102BE000695DD8A0F8EF15F00894089A0EEF16F07A
:102BF0006D0E695DD8A001EF16F00884089A0EEFFB
:102C000016F02D0E695DD8A00AEF16F00894088A18
:102C10000EEF16F00884088A0EEF16F008A813EFDE
:102C200016F018EF16F008A41DEF16F02AEF16F0B4
:102C300008B41DEF16F02AEF16F09251D8B42FEF1A
:102C400016F0922F2FEF16F008A8089608B80886FD
:102C50002FEF16F0010E926F08782FEF16F008AEE6
:102C600034EF16F039EF16F008AA3EEF16F04BEFEE
:102C700016F008BA3EEF16F04BEF16F09351D8B4A9
:102C800050EF16F0932F50EF16F008AE089C08BED8
:102C9000088C50EF16F0010E936F087E50EF16F07F
:102CA00068513F0B010F4F6E372F60EF16F0C80EC3
:102CB000376F0188582F60EF16F0050E586F0686A3
:102CC000C2B260EF16F09E9212004E2A4EA476EF2A
:102CD00016F04E6A02A46FEF16F0020E5D6F02A6A8
:102CE00074EF16F0020E5E6F02840286A19212004B
:102CF000A42B01BA0288018AA1B265EC16F0B2CF0A
:102D000046F1B3CF47F14EC048F1A1B27CEF16F0C7
:102D1000F0901200A92B01BC028A018CA1B265ECD3
:102D200016F0B2CF4FF1B3CF50F14EC051F1A1B276
:102D30008EEF16F0F0921200821CE8AAE896E8BA2C
:102D4000E8860F0B1200FF0E416F426F1200421B0C
:102D5000080E436FD89041334233D8A0B4EF16F039
:102D6000A00E411B010E421B432FAAEF16F01200CA
:102D7000F29EF2BEB8EF16F03DC13CF1F28E009625
:102D800012004AEC17F03250300F5FEC13F0315064
:102D9000300F5FEC13F03050300F5FEC13F02F501A
:102DA000300F5FEC13F02E50300F5FEC13F0120079
:102DB0004AEC17F03050300F5FEC13F02F50300F0B
:102DC0005FEC13F02E50300F5FEC13F01200200E6A
:102DD0005FEC13F0200E5FEC13F0200E5FEC13F0AD
:102DE0001200200E5FEC13F03A0E5FEC13F0200E91
:102DF0005FEC13F012002E502B6E2C6A2F50386EA1
:102E0000396A3A6A3B6A3C6A0A0E3D6E3E6A3F6A1C
:102E1000406A416A11EC18F038502B2639502C22A8
:102E20003050386E396A3A6A3B6A3C6A640E3D6ECD
:102E3000000E3E6E3F6A406A416A11EC18F038504D
:102E40002B2639502C223150386E396A3A6A3B6A47
:102E50003C6AE80E3D6E030E3E6E3F6A406A416A70
:102E600011EC18F038502B2639502C223250386E85
:102E7000396A3A6A3B6A3C6A100E3D6E270E3E6E16
:102E80003F6A406A416A11EC18F038502B263950DD
:102E90002C2212002E6A2F6A306A316A326A100EB2
:102EA0002B5E270E2C5AD8A059EF17F0322A4FEF7D
:102EB00017F0100E2B26270E2C22E80E2B5E030E89
:102EC0002C5AD8A067EF17F0312A5DEF17F0E80E03
:102ED0002B26030E2C22640E2B5E000E2C5AD8A03B
:102EE00075EF17F0302A6BEF17F0640E2B26000EEB
:102EF0002C220A0E2B5ED8A081EF17F02F2A79EF33
:102F000017F00A0E2B242E6E12002E6A2F6A306ADA
:102F1000316A326A336A346A356A800E2B5E960EE5
:102F20002C5A980E2D5AD8A099EF17F0352A8DEF0C
:102F300017F0800E2B26960E2C22980E2D22400E76
:102F40002B5E420E2C5A0F0E2D5AD8A0ABEF17F065
:102F5000342A9FEF17F0400E2B26420E2C220F0E24
:102F60002D22A00E2B5E860E2C5A010E2D5AD8A0B3
:102F7000BDEF17F0332AB1EF17F0A00E2B26860E07
:102F80002C22010E2D22100E2B5E270E2C5A000E25
:102F90002D5AD8A0CFEF17F0322AC3EF17F0100E3A
:102FA0002B26270E2C22E80E2B5E030E2C5AD8A0BF
:102FB000DDEF17F0312AD3EF17F0E80E2B26030EC2
:102FC0002C22640E2B5E000E2C5AD8A0EBEF17F0CB
:102FD000302AE1EF17F0640E2B26000E2C220A0E89
:102FE0002B5ED8A0F7EF17F02F2AEFEF17F00A0E9D
:102FF0002B242E6E12003D5038263E5039223F5071
:103000003A2240503B2241503C2212003D50385E53
:103010003E50395A3F503A5A40503B5A41503C5A20
:1030200012003692369638C042F039C043F03AC0AA
:1030300044F03BC045F03CC046F0386A396A3A6A11
:103040003B6A3C6A280E376E463245324432433280
:103050004232368436A63694D8A0369436B43682B8
:10306000D8B0FBEC17F0D8B03682D8903D363E365B
:103070003F3640364136D8B03686372E24EF18F02A
:10308000120036923D503E103F1040104110D8B40F
:10309000368238C042F039C043F03AC044F03BC0F9
:1030A00045F03CC046F0386A396A3A6A3B6A3C6A85
:1030B000280E376E42364336443645364636383665
:1030C00039363A363B363C3606EC18F03688D8A00E
:1030D0003698D8A0FBEC17F0D88036A8D890372EB9
:1030E0005AEF18F04236433644364536463642C02B
:1030F00038F043C039F044C03AF045C03BF046C018
:103100003CF012008B960000000000000000000060
:103110000000000000000000000000000000948893
:10312000000000000000000000000000000000009F
:1031300000000000000000008B860000000000007E
:10314000000000000000000000000000000000007F
:1031500000008B9894980000000000000000000020
:1031600000000000000000000000000000009B0EB6
:103170001E6E080E1F6E8B960000000000000000FF
:10318000000000000000000000000000000000003F
:103190001E36D8B0DCEF18F08B9894980000000031
:1031A000000000000000000000000000000000001F
:1031B00000000000E9EF18F0948800000000000013
:1031C00000000000000000000000000000000000FF
:1031D00000008B86000000000000000000000000DE
:1031E0000000000000000000000000001F2EBBEFE8
:1031F00018F08B96000000000000000000000000A6
:1032000000000000000000000000000094888B8691
:1032100000000000000000000000000000000000AE
:10322000000000000000000082B867EF26F01200E6
:103230008B9600000000000000000000000000006D
:10324000000000000000000000009488080E1F6EBF
:103250008B8600000000000000000000000000005D
:1032600000000000000000000000D88082A8D89074
:103270001E368B96000000000000000000000000D9
:103280000000000000000000000000001F2E28EFDA
:1032900019F01E508B960000000000000000000096
:1032A00000000000000000000000000000008B98FB
:1032B00094980000000000000000000000000000E2
:1032C000000000000000000000008B8600000000ED
:1032D00000000000000000000000000000000000EE
:1032E0000000000012008B960000000000000000AB
:1032F00000000000000000000000000000000000CE
:103300009488080E1F6E8B860000000000000000ED
:1033100000000000000000000000000000000000AD
:10332000D88082A8D8901E368B960000000000003E
:10333000000000000000000000000000000000008D
:1033400000001F2E83EF19F01E508B960000000026
:10335000000000000000000000000000000000006D
:103360000000000094880000000000000000000041
:1033700000000000000000000000000000008B863C
:10338000000000000000000000000000000000003D
:10339000000000000000000012008B9600000000FA
:1033A000000000000000000000000000000000001D
:1033B00000000000948800000000000000000000F1
:1033C00000000000000000000000000000008B86EC
:1033D00000000000000000000000000000000000ED
:1033E00000000000000000008B989498000000008E
:1033F00000000000000000000000000000000000CD
:1034000000000000850E1E6E080E1F6E8B960000D9
:1034100000000000000000000000000000000000AC
:103420000000000000001E36D8B027EF1AF08B987D
:103430009498000000000000000000000000000060
:103440000000000000000000000034EF1AF0948833
:10345000000000000000000000000000000000006C
:1034600000000000000000008B860000000000004B
:10347000000000000000000000000000000000004C
:1034800000001F2E06EF1AF08B96000000000000CF
:10349000000000000000000000000000000000002C
:1034A000000094888B8600000000000000000000EF
:1034B000000000000000000000000000000082B8D2
:1034C00067EF26F012008B9600000000000000005D
:1034D00000000000000000000000000000000000EC
:1034E0009488080E1F6E8B8600000000000000000C
:1034F00000000000000000000000000000000000CC
:10350000D88082A8D8901E368B960000000000005C
:1035100000000000000000000000000000000000AB
:1035200000001F2E73EF1AF01E508B960000000053
:10353000000000000000000000000000000000008B
:10354000000000008B98949800000000000000002C
:10355000000000000000000000000000000000006B
:103560008B8600000000000000000000000000004A
:103570000000000000000000000012008B96000018
:10358000000000000000000000000000000000003B
:103590000000000000009488080E1F6E8B8600005B
:1035A000000000000000000000000000000000001B
:1035B000000000000000D88082A8D8901E368B96AC
:1035C00000000000000000000000000000000000FB
:1035D00000000000000000001F2ECEEF1AF01E5069
:1035E0008B960000000000000000000000000000BA
:1035F00000000000000000000000948800000000AF
:1036000000000000000000000000000000000000BA
:10361000000000008B860000000000000000000099
:103620000000000000000000000000000000120088
:103630004E0E8B960000000000000000000000000D
:10364000000000000000000000000000948800005E
:10365000000000000000000000000000000000006A
:103660000000000000008B86000000000000000049
:10367000000000000000000000000000000000004A
:103680008B989498000000000000000000000000EB
:103690000000000000000000000000001E6E080E88
:1036A0001F6E8B960000000000000000000000006C
:1036B0000000000000000000000000001E36D8B02E
:1036C00072EF1BF08B98949800000000000000003F
:1036D00000000000000000000000000000000000EA
:1036E0007FEF1BF094880000000000000000000045
:1036F00000000000000000000000000000008B86B9
:1037000000000000000000000000000000000000B9
:1037100000000000000000001F2E51EF1BF08B96F0
:103720000000000000000000000000000000000099
:10373000000000000000000094888B86000000005C
:103740000000000000000000000000000000000079
:103750000000000082B867EF26F012001E6E080E0F
:103760001F6E8B96000000000000000000000000AB
:103770000000000000000000000000001E36D8B06D
:10378000D2EF1BF08B98949800000000000000001E
:103790000000000000000000000000000000000029
:1037A000DFEF1BF094880000000000000000000024
:1037B00000000000000000000000000000008B86F8
:1037C00000000000000000000000000000000000F9
:1037D00000000000000000001F2EB1EF1BF08B96D0
:1037E00000000000000000000000000000000000D9
:1037F000000000000000000094888B86000000009C
:1038000000000000000000000000000000000000B8
:103810000000000082B867EF26F012000F0E1816A5
:103820001950F00B181218501E6E080E1F6E8B9652
:103830000000000000000000000000000000000088
:1038400000000000000000001E36D8B038EF1CF069
:103850008B98949800000000000000000000000019
:1038600000000000000000000000000045EF1CF018
:10387000948800000000000000000000000000002C
:10388000000000000000000000008B860000000027
:103890000000000000000000000000000000000028
:1038A000000000001F2E17EF1CF08B960000000098
:1038B0000000000000000000000000000000000008
:1038C0000000000094888B860000000000000000CB
:1038D00000000000000000000000000000000000E8
:1038E00082B867EF26F01850E8841E6E080E1F6E2F
:1038F0008B960000000000000000000000000000A7
:10390000000000000000000000001E36D8B099EF53
:103910001CF08B989498000000000000000000004C
:103920000000000000000000000000000000A6EF02
:103930001CF094880000000000000000000000005F
:103940000000000000000000000000008B86000066
:103950000000000000000000000000000000000067
:103960000000000000001F2E78EF1CF08B96000076
:103970000000000000000000000000000000000047
:1039800000000000000094888B860000000000000A
:103990000000000000000000000000000000000027
:1039A000000082B867EF26F018501E6E080E1F6EDA
:1039B0008B960000000000000000000000000000E6
:1039C000000000000000000000001E36D8B0F9EF33
:1039D0001CF08B989498000000000000000000008C
:1039E000000000000000000000000000000006EFE2
:1039F0001DF094880000000000000000000000009E
:103A00000000000000000000000000008B860000A5
:103A100000000000000000000000000000000000A6
:103A20000000000000001F2ED8EF1CF08B96000055
:103A30000000000000000000000000000000000086
:103A400000000000000094888B8600000000000049
:103A50000000000000000000000000000000000066
:103A6000000082B867EF26F012000F0E1816193802
:103A7000F00B181218501E6E080E1F6E8B96000069
:103A80000000000000000000000000000000000036
:103A90000000000000001E36D8B05FEF1DF08B98CC
:103AA00094980000000000000000000000000000EA
:103AB000000000000000000000006CEF1DF0948882
:103AC00000000000000000000000000000000000F6
:103AD00000000000000000008B86000000000000D5
:103AE00000000000000000000000000000000000D6
:103AF00000001F2E3EEF1DF08B960000000000001E
:103B000000000000000000000000000000000000B5
:103B1000000094888B860000000000000000000078
:103B2000000000000000000000000000000082B85B
:103B300067EF26F01850E8841E6E080E1F6E8B96F5
:103B40000000000000000000000000000000000075
:103B500000000000000000001E36D8B0C0EF1DF0CD
:103B60008B98949800000000000000000000000006
:103B7000000000000000000000000000CDEF1DF07C
:103B80009488000000000000000000000000000019
:103B9000000000000000000000008B860000000014
:103BA0000000000000000000000000000000000015
:103BB000000000001F2E9FEF1DF08B9600000000FC
:103BC00000000000000000000000000000000000F5
:103BD0000000000094888B860000000000000000B8
:103BE00000000000000000000000000000000000D5
:103BF00082B867EF26F018501E6E080E1F6E8B9667
:103C000000000000000000000000000000000000B4
:103C100000000000000000001E36D8B020EF1EF0AB
:103C20008B98949800000000000000000000000045
:103C30000000000000000000000000002DEF1EF05A
:103C40009488000000000000000000000000000058
:103C5000000000000000000000008B860000000053
:103C60000000000000000000000000000000000054
:103C7000000000001F2EFFEF1DF08B9600000000DB
:103C80000000000000000000000000000000000034
:103C90000000000094888B860000000000000000F7
:103CA0000000000000000000000000000000000014
:103CB00082B867EF26F012008B960000000000002B
:103CC00000000000000000000000000000000000F4
:103CD00000009488000000000000000000000000C8
:103CE0000000000000000000000000008B860000C3
:103CF00000000000000000000000000000000000C4
:103D00000000000000008B98949800000000000064
:103D100000000000000000000000000000000000A3
:103D200000001C341D341E6E1E340E0BA0091E6EC6
:103D3000080E1F6E8B9600000000000000000000BF
:103D400000000000000000000000000000001E361F
:103D5000D8B0BBEF1EF08B989498000000000000D4
:103D60000000000000000000000000000000000053
:103D70000000C8EF1EF09488000000000000000062
:103D80000000000000000000000000000000000033
:103D90008B86000000000000000000000000000012
:103DA000000000000000000000001F2E9AEF1EF02F
:103DB0008B960000000000000000000000000000E2
:103DC0000000000000000000000094888B860000C6
:103DD00000000000000000000000000000000000E3
:103DE00000000000000082B867EF26F01C507F0B37
:103DF0001E6E080E1F6E8B96000000000000000073
:103E000000000000000000000000000000000000B2
:103E10001E36D8B01CEF1FF08B989498000000005D
:103E20000000000000000000000000000000000092
:103E30000000000029EF1FF094880000000000003F
:103E40000000000000000000000000000000000072
:103E500000008B8600000000000000000000000051
:103E60000000000000000000000000001F2EFBEF1B
:103E70001EF08B9600000000000000000000000013
:103E800000000000000000000000000094888B8605
:103E90000000000000000000000000000000000022
:103EA000000000000000000082B867EF26F01B5001
:103EB0001E6E080E1F6E8B960000000000000000B2
:103EC00000000000000000000000000000000000F2
:103ED0001E36D8B07CEF1FF08B989498000000003D
:103EE00000000000000000000000000000000000D2
:103EF0000000000089EF1FF094880000000000001F
:103F000000000000000000000000000000000000B1
:103F100000008B8600000000000000000000000090
:103F20000000000000000000000000001F2E5BEFFA
:103F30001FF08B9600000000000000000000000051
:103F400000000000000000000000000094888B8644
:103F50000000000000000000000000000000000061
:103F6000000000000000000082B867EF26F08B968A
:103F70000000000000000000000000000000000041
:103F80000000000000000000948800000000000015
:103F90000000000000000000000000000000000021
:103FA00000008B8600000000000000000000000000
:103FB0000000000000000000000000008B989498B2
:103FC00000000000000000000000000000000000F1
:103FD00000000000000000001C341D341E6E1E3462
:103FE0000E0BA1091E6E080E1F6E8B9600000000BE
:103FF00000000000000000000000000000000000C1
:10400000000000001E36D8B016EF20F08B98949870
:1040100000000000000000000000000000000000A0
:10402000000000000000000023EF20F09488000052
:104030000000000000000000000000000000000080
:104040000000000000008B8600000000000000005F
:104050000000000000000000000000000000000060
:104060001F2EF5EF1FF08B960000000000000000EF
:104070000000000000000000000000000000000040
:1040800094888B8600000000000000000000000003
:1040900000000000000000000000000082B867EF90
:1040A00026F012008B9600000000000000000000C7
:1040B00000000000000000000000000000009488E4
:1040C00000000000000000000000000000000000F0
:1040D00000000000000000008B86000000000000CF
:1040E00000000000000000000000000000000000D0
:1040F00000008B9894980000000000000000000071
:1041000000000000000000000000000000001C345F
:104110001D341E6E1E340E0BA0091E6E080E1F6E7F
:104120008B9600000000000000000000000000006E
:10413000000000000000000000001E36D8B0B1EF03
:1041400020F08B9894980000000000000000000010
:104150000000000000000000000000000000BEEFB2
:1041600020F0948800000000000000000000000023
:104170000000000000000000000000008B8600002E
:10418000000000000000000000000000000000002F
:104190000000000000001F2E90EF20F08B96000022
:1041A000000000000000000000000000000000000F
:1041B00000000000000094888B86000000000000D2
:1041C00000000000000000000000000000000000EF
:1041D000000082B867EF26F01C507F0B1E6E080EA1
:1041E0001F6E8B9600000000000000000000000021
:1041F0000000000000000000000000001E36D8B0E3
:1042000012EF21F08B98949800000000000000004D
:10421000000000000000000000000000000000009E
:104220001FEF21F094880000000000000000000053
:1042300000000000000000000000000000008B866D
:10424000000000000000000000000000000000006E
:1042500000000000000000001F2EF1EF20F08B9600
:10426000000000000000000000000000000000004E
:10427000000000000000000094888B860000000011
:10428000000000000000000000000000000000002E
:104290000000000082B867EF26F01B501E6E080E6B
:1042A0001F6E8B9600000000000000000000000060
:1042B0000000000000000000000000001E36D8B022
:1042C00072EF21F08B98949800000000000000002D
:1042D00000000000000000000000000000000000DE
:1042E0007FEF21F094880000000000000000000033
:1042F00000000000000000000000000000008B86AD
:1043000000000000000000000000000000000000AD
:1043100000000000000000001F2E51EF21F08B96DE
:10432000000000000000000000000000000000008D
:10433000000000000000000094888B860000000050
:10434000000000000000000000000000000000006D
:104350000000000082B867EF26F012001E6E080E03
:104360001F6E8B960000000000000000000000009F
:104370000000000000000000000000001E36D8B061
:10438000D2EF21F08B98949800000000000000000C
:10439000000000000000000000000000000000001D
:1043A000DFEF21F094880000000000000000000012
:1043B00000000000000000000000000000008B86EC
:1043C00000000000000000000000000000000000ED
:1043D00000000000000000001F2EB1EF21F08B96BE
:1043E00000000000000000000000000000000000CD
:1043F000000000000000000094888B860000000090
:1044000000000000000000000000000000000000AC
:104410000000000082B867EF26F012008B960000C3
:10442000000000000000000000000000000000008C
:104430000000000000009488080E1F6E8B860000AC
:10444000000000000000000000000000000000006C
:10445000000000000000D88082A8D8901E368B96FD
:10446000000000000000000000000000000000004C
:1044700000000000000000001F2E1EEF22F01E5062
:104480008B9600000000000000000000000000000B
:10449000000000000000000000008B9894980000CD
:1044A000000000000000000000000000000000000C
:1044B0000000000000008B860000000000000000EB
:1044C00000000000000000000000000000000000EC
:1044D00012008B96000000000000000000000000A9
:1044E0000000000000000000000000009488080E9A
:1044F0001F6E8B860000000000000000000000001E
:10450000000000000000000000000000D88082A829
:10451000D8901E368B9600000000000000000000BE
:1045200000000000000000000000000000001F2E3E
:1045300079EF22F01E508B96000000000000000072
:10454000000000000000000000000000000000006B
:10455000948800000000000000000000000000003F
:10456000000000000000000000008B86000000003A
:10457000000000000000000000000000000000003B
:10458000000000001200196E18900EEC1CF035ECC3
:104590001DF012001880196E0EEC1CF035EC1DF0A9
:1045A00012008B96000000000000000000000000D8
:1045B00000000000000000000000000094880000DF
:1045C00000000000000000000000000000000000EB
:1045D0000000000000008B860000000000000000CA
:1045E00000000000000000000000000000000000CB
:1045F0008B9894980000000000000000000000006C
:10460000000000000000000000000000A00E1E6E70
:10461000080E1F6E8B9600000000000000000000D6
:1046200000000000000000000000000000001E3636
:10463000D8B02BEF23F08B98949800000000000076
:10464000000000000000000000000000000000006A
:10465000000038EF23F09488000000000000000004
:10466000000000000000000000000000000000004A
:104670008B86000000000000000000000000000029
:10468000000000000000000000001F2E0AEF23F0D1
:104690008B960000000000000000000000000000F9
:1046A0000000000000000000000094888B860000DD
:1046B00000000000000000000000000000000000FA
:1046C00000000000000082B867EF26F01B501E6E4D
:1046D000080E1F6E8B960000000000000000000016
:1046E00000000000000000000000000000001E3676
:1046F000D8B08BEF23F08B98949800000000000056
:1047000000000000000000000000000000000000A9
:10471000000098EF23F094880000000000000000E3
:104720000000000000000000000000000000000089
:104730008B86000000000000000000000000000068
:10474000000000000000000000001F2E6AEF23F0B0
:104750008B96000000000000000000000000000038
:104760000000000000000000000094888B8600001C
:104770000000000000000000000000000000000039
:1047800000000000000082B867EF26F08B96000062
:104790000000000000000000000000000000000019
:1047A00000000000000094880000000000000000ED
:1047B00000000000000000000000000000000000F9
:1047C0008B860000000000000000000000000000D8
:1047D000000000000000000000008B98949800008A
:1047E00000000000000000000000000000000000C9
:1047F000000000000000A10E1E6E080E1F6E8B96BA
:1048000000000000000000000000000000000000A8
:1048100000000000000000001E36D8B020EF24F099
:104820008B98949800000000000000000000000039
:104830000000000000000000000000002DEF24F048
:10484000948800000000000000000000000000004C
:10485000000000000000000000008B860000000047
:104860000000000000000000000000000000000048
:10487000000000001F2EFFEF23F08B9600000000C9
:104880000000000000000000000000000000000028
:104890000000000094888B860000000000000000EB
:1048A0000000000000000000000000000000000008
:1048B00082B867EF26F012008B960000000000001F
:1048C00000000000000000000000000000000000E8
:1048D00000009488000000000000000000000000BC
:1048E0000000000000000000000000008B860000B7
:1048F00000000000000000000000000000000000B8
:104900000000000000008B98949800000000000058
:104910000000000000000000000000000000000097
:104920000000A00E1E6E080E1F6E8B960000000089
:104930000000000000000000000000000000000077
:10494000000000001E36D8B0B6EF24F08B98949883
:104950000000000000000000000000000000000057
:104960000000000000000000C3EF24F09488000065
:104970000000000000000000000000000000000037
:104980000000000000008B86000000000000000016
:104990000000000000000000000000000000000017
:1049A0001F2E95EF24F08B96000000000000000001
:1049B00000000000000000000000000000000000F7
:1049C00094888B86000000000000000000000000BA
:1049D00000000000000000000000000082B867EF47
:1049E00026F01B501E6E080E1F6E8B9600000000F6
:1049F00000000000000000000000000000000000B7
:104A0000000000001E36D8B016EF25F08B98949861
:104A10000000000000000000000000000000000096
:104A2000000000000000000023EF25F09488000043
:104A30000000000000000000000000000000000076
:104A40000000000000008B86000000000000000055
:104A50000000000000000000000000000000000056
:104A60001F2EF5EF24F08B960000000000000000E0
:104A70000000000000000000000000000000000036
:104A800094888B86000000000000000000000000F9
:104A900000000000000000000000000082B867EF86
:104AA00026F012001E6E080E1F6E8B96000000008E
:104AB00000000000000000000000000000000000F6
:104AC000000000001E36D8B076EF25F08B98949841
:104AD00000000000000000000000000000000000D6
:104AE000000000000000000083EF25F09488000023
:104AF00000000000000000000000000000000000B6
:104B00000000000000008B86000000000000000094
:104B10000000000000000000000000000000000095
:104B20001F2E55EF25F08B960000000000000000BE
:104B30000000000000000000000000000000000075
:104B400094888B8600000000000000000000000038
:104B500000000000000000000000000082B867EFC5
:104B600026F012008B9600000000000000000000FC
:104B70000000000000000000000000000000948819
:104B8000080E1F6E8B860000000000000000000071
:104B90000000000000000000000000000000D880BD
:104BA00082A8D8901E368B960000000000000000FE
:104BB00000000000000000000000000000000000F5
:104BC0001F2EC2EF25F01E508B9600000000000043
:104BD00000000000000000000000000000000000D5
:104BE00000008B9894980000000000000000000076
:104BF00000000000000000000000000000008B86A4
:104C000000000000000000000000000000000000A4
:104C1000000000000000000012008B960000000061
:104C20000000000000000000000000000000000084
:104C3000000000009488080E1F6E8B8600000000A4
:104C40000000000000000000000000000000000064
:104C500000000000D88082A8D8901E368B960000F5
:104C60000000000000000000000000000000000044
:104C70000000000000001F2E1DEF26F01E508B9636
:104C80000000000000000000000000000000000024
:104C900000000000000000009488000000000000F8
:104CA0000000000000000000000000000000000004
:104CB00000008B86000000000000000000000000E3
:104CC000000000000000000000000000120005804D
:104CD0008B960000000000000000000000000000B3
:104CE000000000000000000000008B989498000075
:104CF00000000000000000000000000000000000B4
:104D00000000000000008B86000000000000000092
:104D10000000000000000000000000000000000093
:104D20009488000000000000000000000000000067
:104D30000000000000000000000012000000000061
:104D40008B96000000000000000000000000000042
:104D5000000000000000000000008B989498000004
:104D60000000000000000000000000000000000043
:104D70000000000000008B86000000000000000022
:104D80000000000000000000000000000000000023
:104D900094880000000000000000000000000000F7
:104DA000000000000000000000001200096E093839
:104DB000E1EC26F00950E1EC26F0200E5FEC13F058
:104DC00012000F0B0A6E0A0E0A5C300ED8B0370EB6
:104DD0000A245FEC13F01200C26EC282C2B2EEEF80
:104DE00026F012000588F8EF26F00598F8EF26F077
:104DF0000900F550D8B401EF27F05FEC13F0F8EF9D
:104E000026F005881200800EC3EC22F0B4EC12F0FC
:104E10000900F550D8B411EF27F0CAEC22F008EFE2
:104E200027F01200C00EC3EC22F0B4EC12F009001F
:104E3000F550D8B420EF27F0CAEC22F017EF27F096
:104E40001200B751C3EC22F0B4EC12F04AEC17F0A8
:104E50003250300FCAEC22F03150300FCAEC22F041
:104E60003050300FCAEC22F02F50300FCAEC22F035
:104E70002E50300FCAEC22F01200B751C3EC22F0D2
:104E8000B4EC12F04AEC17F03150300FCAEC22F0BB
:104E90003050300FCAEC22F02F50300FCAEC22F005
:104EA0002E50300FCAEC22F012004F0E5FEC13F0C0
:104EB000410E5FEC13F0320E5FEC13F0390E5FEC35
:104EC00013F012000D0E5FEC13F00A0E5FEC13F0FE
:104ED000120001AA99EF27F0F29E019A46C149F10A
:104EE00047C14AF148C14BF1029402804C51495DDF
:104EF000A56F4D514A59A66F4E514B59A76F49C1E5
:104F00004CF14AC14DF14BC14EF15D51D8B48FEF18
:104F100027F05D07FF0EA46BA56FA66FA76F030EAA
:104F2000A7B5A717F28E33EC0DF0C80EB86F000EC0
:104F3000B96F120001ACC3EF27F0F29E019C4FC184
:104F400052F150C153F151C154F1029602825551B0
:104F5000525DAA6F56515359AB6F57515459030BB9
:104F6000AC6F52C155F153C156F154C157F15E5166
:104F7000D8B4C3EF27F05E07FF0EA96BAA6FAB6F23
:104F8000AC6FC3EF27F0F28E120002AC48EF29F0AD
:104F9000029C5F51000AD8B4DCEF27F0010AD8B4B4
:104FA00033EF28F0030AD8B4E5EF28F0010AD8B4AB
:104FB000E7EF28F00CEF29F04D50D8A4EAEF27F0E6
:104FC000280E4D6EA68EF86A090EF76E220EF66E4A
:104FD000F2EC26F0B1C12BF02C6AD8EC16F0F1EC13
:104FE00016F0A1C12BF0A2C12CF0C1EC16F0F1EC2F
:104FF00016F0F29E99C12BF09AC12CF0F28EC1EC02
:1050000016F0F1EC16F0F29E90C1E9FF91C1EAFFB3
:10501000EECFE8FFEECF2BF0EECF2CF0F28EC1EC0E
:1050200016F0F1EC16F0C1EC16F00588F1EC16F074
:10503000450E5FEC13F03D0E5FEC13F0300E310EB9
:105040005FEC13F0F1EC16F0520E5FEC13F03D0E36
:105050005FEC13F07F0B300F5FEC13F0059862EC00
:1050600027F048EF29F0B1C12BF02C6AD8EC16F0EC
:10507000F1EC16F0B2C12BF02C6AD8EC16F0F1EC82
:1050800016F001EE00F0EECFE8FFD6EC26F0EECF02
:10509000E8FFD6EC26F0EECFE8FFD6EC26F0280E9F
:1050A0005FEC13F0300E02B5310E5FEC13F0300EF2
:1050B00002B3310E5FEC13F0300E02B1310E5FEC33
:1050C00013F0290E5FEC13F0200E5FEC13F0EECF1F
:1050D000E8FFD6EC26F0EECFE8FFD6EC26F0EECFD8
:1050E000E8FFD6EC26F0EECFE8FFD6EC26F0EECFC8
:1050F000E8FFD6EC26F0EECFE8FFD6EC26F0EECFB8
:10510000E8FFD6EC26F0EECFE8FFD6EC26F0EECFA7
:10511000E8FFD6EC26F0EECFE8FFD6EC26F0EECF97
:10512000E8FFD6EC26F0EECFE8FFD6EC26F0EECF87
:10513000E8FFD6EC26F03A0E5FEC13F0200E5FECA1
:1051400013F0EECFE8FFD6EC26F0EECFE8FFD6EC7A
:1051500026F0EECFE8FFD6EC26F0EECFE8FFD6EC57
:1051600026F0EECFE8FFD6EC26F0EECFE8FFD6EC47
:1051700026F0EECFE8FFD6EC26F0EECFE8FFD6EC37
:1051800026F0EECFE8FFD6EC26F0EECFE8FFD6EC27
:1051900026F0EECFE8FFD6EC26F0EECFE8FFD6EC17
:1051A00026F0EECFE8FFD6EC26F0EECFE8FFD6EC07
:1051B00026F0EECFE8FFD6EC26F0EECFE8FFD6ECF7
:1051C00026F062EC27F048EF29F048EF29F04D5027
:1051D000D8A4F7EF28F0280E4D6EA68EF86A090EB7
:1051E000F76E0E0EF66EF2EC26F00AEF29F0B1C162
:1051F0002BF02C6AD8EC16F0F1EC16F02C6AD8ECF7
:1052000016F0F1EC16F09CC12BF02C6AD8EC16F0DD
:1052100062EC27F048EF29F04D50D8A41CEF29F09C
:10522000280E4D6EA68EF86A090EF76E4A0EF66EBF
:10523000F2EC26F048EF29F002A048EF29F00290A6
:10524000AAC12BF0ABC100F085EC17F03550300F40
:105250005FEC13F03450300F5FEC13F03350300F2D
:105260005FEC13F03250300F5FEC13F03150300F21
:105270005FEC13F03050300F5FEC13F02F50300F15
:105280005FEC13F02E50300F5FEC13F062EC27F060
:10529000120008BC51EF29F02B502C10D8B478EF35
:1052A00029F02B50995D386E2C509A59396ED8A040
:1052B00067EF29F05CEF29F08A98640E385C000EE5
:1052C0003958010ED8B0190E276E78EF29F08A8868
:1052D000381E391E010E3826000E3922640E385C45
:1052E000000E3958010ED8B0190E276E78EF29F04C
:1052F0001200F29EF2BE79EF29F039C138F1F28E38
:10530000120038513919D8A4D880D8B4D890D8B45C
:105310009CEF29F091EF29F038513919D8B48CEF6E
:1053200029F023EE00F03829FA0AD8B4FA0EFA0A66
:10533000D96E386FDF50D88012003C513D19D8A487
:10534000D880D8B4D890D8B4B8EF29F0ADEF29F010
:105350003C513D19D8B4A8EF29F022EE40F03C2989
:10536000800AD8B4C00E800AD96E3C6FDF50D88056
:1053700012003491FA0E556E000E546E120081EC3C
:1053800029F0D8A007EF2AF0566E5550D8B4DCEFBC
:1053900029F024EE00F05450D96E542A5650DF6E96
:1053A00055060D0AD8B4DCEF29F0070AD8B4DCEFB3
:1053B00029F0BFEF29F0348324EE00F0FA0E576E87
:1053C0005550575E572EE9EF29F0B9EC29F0BFEFA1
:1053D00029F0DF50349508EC2AF034A5F4EF29F0D9
:1053E000B9EC29F0BFEF29F020EC2AF0A68EF86A7C
:1053F000060EF76E800EF66E140E5C6E5DEC2AF0F3
:10540000D8B005EF2AF0FF0E5A6E5A5034811200C0
:1054100034B51BEF2AF0DF50200AD8B416EF2AF07B
:10542000290AD8B416EF2AF01BEF2AF0D92A572EF2
:1054300008EF2AF03485D950586E596ADF501200AF
:1054400034B52EEF2AF0ACEC2AF0D8A02EEF2AF0DB
:10545000D92A592A572E20EF2AF03485DF50595285
:10546000120034B53FEF2AF003EC2BF0D8A03FEF49
:105470002AF0D92A592A572E31EF2AF03485DF50E5
:105480005952120034B550EF2AF029EC2BF0D8A075
:1054900050EF2AF0D92A592A572E42EF2AF03485A4
:1054A000DF505952120034B55BEF2AF0D92A572E3B
:1054B0005BEF2AF03485DF5012005950D8B48BEFDF
:1054C0002AF05A6A5850D96E59505B6E0900F5504F
:1054D000FF0BD8B480EF2AF0DF5CD8A47AEF2AF073
:1054E000D92A5B2E66EF2AF00900F550FF0BD8B4DD
:1054F0008EEF2AF00900F550FF0BD8A47AEF2AF0BE
:105500000900F550FF0BD8B480EF2AF00A005A2AA0
:105510005C2E62EF2AF0D8908FEF2AF0D88012002C
:10552000410EDF5CD8A0A9EF2AF05B0EDF5CD8A0AB
:10553000A6EF2AF0610EDF5CD8A0A9EF2AF07B0E5F
:10554000DF5CD8B0A9EF2AF0200EDF5ED880AAEF8A
:105550002AF0D890DF501200200EDF5C34ABD894D4
:10556000D8B4FDEF2AF0210EDF5CD8B4FDEF2AF0AD
:10557000220E34A9230EDF5CD8A000EF2BF02C0EF6
:10558000DF5CD8A0FDEF2AF02C0E34AB2D0EDF5CD3
:10559000D8A000EF2BF0300EDF5CD8A0FDEF2AF092
:1055A000300EDF5CD8A000EF2BF03A0EDF5CD8A005
:1055B000FDEF2AF03A0EDF5CD8A000EF2BF0410E91
:1055C000DF5CD8A0FDEF2AF0410EDF5CD8A000EF31
:1055D0002BF05B0EDF5CD8A0FDEF2AF0610EDF5CE4
:1055E000D8A000EF2BF07B0EDF5CD8B000EF2BF0E3
:1055F00034A7FDEF2AF0200EDF5ED88001EF2BF0FC
:10560000D890DF501200300EDF5CD8A026EF2BF0D0
:105610003A0EDF5CD8A023EF2BF0410EDF5CD8A060
:1056200026EF2BF05B0EDF5CD8A023EF2BF0610E92
:10563000DF5CD8A026EF2BF07B0EDF5CD8B026EF26
:105640002BF0200EDF5ED88027EF2BF0D890DF50B4
:105650001200300EDF5CD8A036EF2BF03A0EDF5C84
:10566000D8B036EF2BF0D88037EF2BF0D890DF5042
:105670001200BB6FBB3945EC2BF04BEC13F0BB5168
:1056800045EC2BF04BEC13F012000F0B300FBA6F00
:105690003A0EBA5D070ED8A0000EBA251200FB6ABA
:1056A000BCC1BDF1BE6BD890BD37BE37BD37BE376C
:1056B000BE0EBD27560EBE21FA6EBD51F96ECBEF60
:1056C0002BF0D3EF2BF0DCEF2BF0F1EF2BF0FCEF16
:1056D0002BF004EF2CF00BEF2CF022EF2CF038EF36
:1056E0002CF055EF2CF064EF2CF07DEF2CF090EFC8
:1056F0002CF0ABEF2CF0B2EF2CF0CBEF2CF0DEEF78
:105700002CF0EDEF2CF0F4EF2CF00DEF2DF020EF5E
:105710002DF02FEF2DF036EF2DF04FEF2DF062EF43
:105720002DF068EF2EF06FEF2EF086EF2EF099EF50
:105730002EF0A9EF2EF0B0EF2EF0C7EF2EF0DAEF3B
:105740002EF0F3EF2EF0FAEF2EF011EF2FF024EF02
:105750002FF086EF2FF09BEF2FF0DAEF2FF0E1EF35
:105760002FF00DEF30F02BEF30F0CFEF30F0E2EF15
:1057700030F0FCEF30F003EF31F033EF31F046EF73
:1057800031F057EF31F06AEF31F075EF31F087EF1C
:1057900031F08CEF31F0050E586F010EE8CFBCF1FF
:1057A00006964FEF2BF006A6DAEF2BF00696050EC5
:1057B000E8CFBCF1A0EF31F080B2E7EF2BF08980A9
:1057C000A1EC31F0030EE8CFBCF1A0EF31F08990ED
:1057D000C5EC31F0040EE8CFBCF11E0E5F6EA0EFF9
:1057E00031F034ADFAEF2BF08990C5EC31F0040EB6
:1057F000E8CFBCF1A0EF31F034AD02EF2CF0050E94
:10580000E8CFBCF1A0EF31F0B3EC31F0060EE8CFF9
:10581000BCF1A0EF31F034AD20EF2CF079EC29F0A1
:10582000349FA68EF86A040EF76E000EF66E07EC33
:1058300032F0B9EC31F0B9EC29F0070EE8CFBCF149
:10584000A0EF31F0348BBFEC29F034A12DEF2CF018
:10585000080EE8CFBCF14FEF2BF034AD36EF2CF053
:105860003591310E89A0020EE8CFBCF1A0EF31F0E6
:105870005A50010AD8A445EF2CF03583B9EC29F031
:10588000070EE8CFBCF14FEF2BF0010AD8A44FEF81
:105890002CF03581090EE8CFBCF153EF2CF0359197
:1058A000310EE8CFBCF1A0EF31F035B35DEF2CF055
:1058B0000D0EE8CFBCF162EF2CF0B3EC31F00A0E24
:1058C000E8CFBCF1A0EF31F034AD7BEF2CF079ECF8
:1058D00029F0349FA68EF86A040EF76E040EF66E59
:1058E00007EC32F0B9EC31F0B9EC29F00B0EE8CF4F
:1058F000BCF14FEF2BF0A0EF31F0348BBFEC29F06F
:1059000034A188EF2CF00C0EE8CFBCF14FEF2BF058
:1059100034AD8EEF2CF0310EE8CFBCF1A0EF31F0BA
:105920005A50020AD8A49CEF2CF0B9EC29F00B0EC7
:10593000E8CFBCF14FEF2BF0020AD8A4A6EF2CF071
:1059400035930D0EE8CFBCF1A9EF2CF0310EE8CF66
:10595000BCF1A0EF31F0B3EC31F00E0EE8CFBCF1AA
:10596000A0EF31F034ADC9EF2CF079EC29F0349F81
:10597000A68EF86A040EF76E0A0EF66E07EC32F089
:10598000B9EC31F0B9EC29F00F0EE8CFBCF14FEFD4
:105990002BF0A0EF31F0348BBFEC29F034A1D6EF1F
:1059A0002CF0100EE8CFBCF14FEF2BF034ADDCEF54
:1059B0002CF0310EE8CFBCF1A0EF31F05A50000AC4
:1059C000D8A4E8EF2CF0110EE8CFBCF14FEF2BF08C
:1059D000110EE8CFBCF1A0EF31F0B3EC31F0120EB4
:1059E000E8CFBCF1A0EF31F034AD0BEF2DF079EC46
:1059F00029F0349FA68EF86A040EF76E160EF66E26
:105A000007EC32F0B9EC31F0B9EC29F0130EE8CF25
:105A1000BCF14FEF2BF0A0EF31F0348BBFEC29F04D
:105A200034A118EF2DF0140EE8CFBCF14FEF2BF09E
:105A300034AD1EEF2DF0310EE8CFBCF1A0EF31F008
:105A40005A50000AD8A42AEF2DF0150EE8CFBCF169
:105A50004FEF2BF0150EE8CFBCF1A0EF31F0B3EC17
:105A600031F0160EE8CFBCF1A0EF31F034AD4DEFC0
:105A70002DF079EC29F0349FA68EF86A040EF76EAB
:105A80001C0EF66E07EC32F0B9EC31F0B9EC29F0EF
:105A9000170EE8CFBCF14FEF2BF0A0EF31F0349BA5
:105AA000BFEC29F034A15AEF2DF0180EE8CFBCF16D
:105AB0004FEF2BF034AD60EF2DF0310EE8CFBCF19D
:105AC000A0EF31F05A50000AD8A46CEF2DF0190E57
:105AD000E8CFBCF14FEF2BF05A50120AD8A463EF75
:105AE0002EF0190EE8CFBCF108EC2AF0220EDF5C94
:105AF000D8A45AEF2EF053EC2AF029EC2BF0D8A0C2
:105B00005AEF2EF0300EDF5CE838CF6F53EC2AF0FE
:105B100029EC2BF0D8A05AEF2EF0300EDF5CCF131B
:105B200053EC2AF02F0EDF5CD8A45AEF2EF053EC82
:105B30002AF029EC2BF0D8A05AEF2EF0300EDF5CC3
:105B4000E838CE6F53EC2AF029EC2BF0D8A05AEFAE
:105B50002EF0300EDF5CCE1353EC2AF02F0EDF5CFC
:105B6000D8A45AEF2EF053EC2AF029EC2BF0D8A051
:105B70005AEF2EF0300EDF5CE838CD6F53EC2AF090
:105B800029EC2BF0D8A05AEF2EF0300EDF5CCD13AD
:105B900053EC2AF02C0EDF5CD8A45AEF2EF053EC15
:105BA0002AF029EC2BF0D8A05AEF2EF0300EDF5C53
:105BB000E838CC6F53EC2AF029EC2BF0D8A05AEF40
:105BC0002EF0300EDF5CCC1353EC2AF03A0EDF5C83
:105BD000D8A45AEF2EF053EC2AF029EC2BF0D8A0E1
:105BE0005AEF2EF0300EDF5CE838CB6F53EC2AF022
:105BF00029EC2BF0D8A05AEF2EF0300EDF5CCB133F
:105C000053EC2AF03A0EDF5CD8A45AEF2EF053EC96
:105C10002AF029EC2BF0D8A05AEF2EF0300EDF5CE2
:105C2000E838CA6F53EC2AF029EC2BF0D8A05AEFD1
:105C30002EF0300EDF5CCA1353EC2AF0D06F53EC19
:105C40002AF029EC2BF0D8A05AEF2EF0300EDF5CB2
:105C5000D16F53EC2AF029EC2BF0D8A05AEF2EF09C
:105C6000300EDF5CD26FCF51C819D8A45AEF2EF096
:105C7000CE51C719D8A45AEF2EF0CD51C619D8A4C9
:105C80005AEF2EF0CC51C419D8A45AEF2EF0CB51B4
:105C9000C35DD8B04EEF2EF0C351CB5D000AD8B42F
:105CA0005AEF2EF0010AD8B45AEF2EF0030AD8B4F6
:105CB0005AEF2EF0BDEC12F0B9EC29F0170EE8CF38
:105CC000BCF14FEF2BF01D0EE8CFBCF1A0EF31F08F
:105CD000B3EC31F01A0EE8CFBCF1A0EF31F034ADE7
:105CE00084EF2EF079EC29F0349FA68EF86A040E2A
:105CF000F76E260EF66E07EC32F0B9EC31F0B9EC27
:105D000029F01B0EE8CFBCF1A0EF31F0348BBFECD3
:105D100029F034A191EF2EF01C0EE8CFBCF14FEF2B
:105D20002BF034AD97EF2EF0310EE8CFBCF1A0EFA1
:105D300031F05A50000AD8A4A4EF2EF0C16B1D0E0A
:105D4000E8CFBCF1A7EF2EF0310EE8CFBCF1A0EF09
:105D500031F0DBEC31F01E0EE8CFBCF1A0EF31F0FA
:105D600034ADC5EF2EF079EC29F0349FA68EF86A99
:105D7000040EF76E320EF66E07EC32F0B9EC31F02D
:105D8000B9EC29F01F0EE8CFBCF1A0EF31F0348B55
:105D9000BFEC29F034A1D2EF2EF0200EE8CFBCF1F9
:105DA0004FEF2BF034ADD8EF2EF0310EE8CFBCF131
:105DB000A0EF31F05A50040AD8A4E4EF2EF0210EDF
:105DC000E8CFBCF1F1EF2EF05A50050AD8A4EEEF5F
:105DD0002EF0270EE8CFBCF1F1EF2EF0310EE8CF18
:105DE000BCF1A0EF31F0B9EC31F0220EE8CFBCF1FC
:105DF000A0EF31F034AD0FEF2FF079EC29F0349FA4
:105E0000A68EF86A040EF76EBE0EF66E07EC32F040
:105E1000BFEC31F0B9EC29F0230EE8CFBCF1A0EFD4
:105E200031F0349BBFEC29F034A11CEF2FF0240E8D
:105E3000E8CFBCF14FEF2BF034AD22EF2FF0310E55
:105E4000E8CFBCF1A0EF31F05A50000AD8A431EFEE
:105E50002FF05F06000ED8B4310EE8CFBCF184EF0E
:105E60002FF05A500B0AD8B43CEF2FF00694310EA5
:105E7000E8CFBCF184EF2FF01E0E5F6E08EC2AF025
:105E800042EC2AF0D9CFE9FFDACFEAFFD66BDD503A
:105E9000010ED76FDD50D00FD703F350D6270A0E6F
:105EA000D703F3CFD7F1592E4AEF2FF0E9CFD9FF1F
:105EB000EACFDAFFD86B34B57FEF2FF053EC2AF03E
:105EC0002C0AD8A45BEF2FF034B57FEF2FF053EC02
:105ED0002AF0220AD8A47FEF2FF001EED9F034B5D2
:105EE0007EEF2FF053EC2AF0220AD8B47FEF2FF088
:105EF000220AEE6ED82BD8A96FEF2FF0D86BB9EC31
:105F000029F0250EE8CFBCF1A0EF31F0348B3497A7
:105F1000BFEC29F0348734A193EF2FF0260EE8CFA1
:105F2000BCF14FEF2BF034AD99EF2FF0000EE8CF1E
:105F3000BCF1A0EF31F0069224EE00F0D906F90E84
:105F4000576E5550575E349534B5D0EF2FF053EC63
:105F50002AF0EA19D8A4D0EF2FF034B5D0EF2FF003
:105F600053EC2AF0EB19D8A4D0EF2FF034B5D0EFD2
:105F70002FF053EC2AF0EC19D8A4D0EF2FF034B561
:105F8000D0EF2FF053EC2AF0ED19D8A4D0EF2FF07A
:105F9000068234B5D0EF2FF053EC2AF0D0EF2FF07B
:105FA000270E06A22D0ED853D8B42D0EE8CFBCF183
:105FB000A0EF31F0B3EC31F0280EE8CFBCF1A0EF48
:105FC00031F081EC29F0D8A0E8EF2FF0B3EC31F0FC
:105FD00034AD0BEF30F079EC29F0348FA68EF86AEF
:105FE000040EF76E3C0EF66E07EC32F001EED9F0BF
:105FF000D8C1D3F1EE504BEC13F0D32FFAEF2FF0C2
:10600000220E4BEC13F00D0E4BEC13F0B9EC31F00B
:10601000290EE8CFBCF1A0EF31F081EC29F0D8A037
:1060200023EF30F00D0AD8B40DEF30F0070AD8B4E2
:106030000DEF30F0340AD8A426EF30F02A0EE8CF66
:10604000BCF129EF30F034AD29EF30F0310EE8CF5C
:10605000BCF1A0EF31F081EC29F0D8A0C7EF30F00F
:10606000200AD8A4CAEF30F0348FA68EF86A040E46
:10607000F76E580EF66E07EC32F0F5C12BF0F6C154
:106080002CF04AEC17F03250300F4BEC13F031503B
:10609000300F4BEC13F03050300F4BEC13F02F500F
:1060A000300F4BEC13F02E50300F4BEC13F0200E52
:1060B0004BEC13F06F0E4BEC13F0660E4BEC13F041
:1060C000200E4BEC13F099C12BF09AC12CF04AEC46
:1060D00017F03250300F4BEC13F03150300F4BECC7
:1060E00013F03050300F4BEC13F02F50300F4BECBF
:1060F00013F02E50300F4BEC13F0200E4BEC13F03E
:106100004C0E4BEC13F02F0E4BEC13F0480E4BECF7
:1061100013F007A08EEF30F098EF30F0A68EF86AFB
:10612000040EF76E6C0EF66E07EC32F0A2EF30F054
:10613000A68EF86A040EF76E7E0EF66E07EC32F04D
:10614000A2EF30F007A2A7EF30F0B1EF30F0A68E4B
:10615000F86A040EF76EA60EF66E07EC32F0BBEF8F
:1061600030F0A68EF86A040EF76E8E0EF66E07EC0F
:1061700032F0BBEF30F01A0E4BEC13F018EC32F0AB
:10618000B9EC29F02B0EE8CFBCF1CDEF30F034ADF7
:10619000CDEF30F0310EE8CFBCF1A0EF31F0349B01
:1061A000BFEC29F034A1DAEF30F02C0EE8CFBCF1CF
:1061B0004FEF2BF034ADE0EF30F0310EE8CFBCF113
:1061C000A0EF31F05A500A0AD8A4EEEF30F0B9EC43
:1061D00029F02B0EE8CFBCF1FAEF30F00A0AD8A470
:1061E000F7EF30F02D0EE8CFBCF1FAEF30F02D0EC6
:1061F000E8CFBCF1A0EF31F0BFEC31F02E0EE8CFCC
:10620000BCF1A0EF31F034AD31EF31F0D76B0A0EB5
:10621000D65FD8A00FEF31F0D72B08EF31F0D6279B
:1062200079EC29F0348FA68EF86A040EF76ED80E3A
:10623000F66E07EC32F0349FD751D8B423EF31F02B
:10624000300F4BEC13F0D651300F4BEC13F00D0E1A
:106250004BEC13F0B9EC31F0B9EC29F02F0EE8CF8C
:10626000BCF1A0EF31F0349BBFEC29F034A13EEF3C
:1062700031F0300EE8CFBCF14FEF2BF034AD44EFEE
:1062800031F0310EE8CFBCF1A0EF31F05A50000AE6
:10629000D8A450EF31F0000EE8CFBCF155EF31F04B
:1062A000310EE8CFBCF155EF31F0A0EF31F080A214
:1062B00062EF31F08980A7EC31F0320EE8CFBCF10B
:1062C000A0EF31F08990B9EC31F0350EE8CFBCF198
:1062D000A0EF31F034ADFAEF2BF08990ADEC31F056
:1062E000330EE8CFBCF1A0EF31F034AD7DEF31F0EB
:1062F000310EE8CFBCF185EF31F080B285EF31F09F
:10630000350E06A0340EE8CFBCF1A0EF31F0000E40
:10631000E8CFBCF1A0EF31F034AD9EEF31F0E851A1
:10632000D8B499EF31F0E807020EE8CFBCF19EEF48
:1063300031F0000EE8CFBCF19EEF31F0A0EF31F06C
:106340001200C80EBF6F000EC06F349D1200A40E65
:10635000BF6F010EC06F349D1200280EBF6F000E7C
:10636000C06F349D1200140EBF6F000EC06F349DBD
:106370001200E80EBF6F030EC06F349D1200D00EE6
:10638000BF6F070EC06F349D1200F29EF2BEC5EFC4
:1063900031F0A00EBF6F0F0EC06F349DF28E120051
:1063A000F29EF2BED0EF31F0500EBF6F460EC06FBE
:1063B000349DF28E1200F29EF2BEDBEF31F0E80E59
:1063C000BF6F030EC06F349DF28E1200F29EF2BEBC
:1063D000E6EF31F0E00EBF6F2E0EC06F349DF28EEF
:1063E0001200F29EF2BEF1EF31F0980EBF6F3A0E3E
:1063F000C06F349DF28E1200F29EF2BEFCEF31F0BF
:10640000680EBF6F420EC06F349DF28E12000900FD
:10641000F550FF0BD8B411EF32F04BEC13F007EF4F
:1064200032F034BF17EF32F00D0E4BEC13F01200C8
:10643000A00EBF6F8C0EC06F349D120006EE00F0F0
:10644000E950C00F0EEC00F0EE6EE9AC20EF32F038
:106450001200FFFFFFFFFFFFFFFFFFFFFFFFFFFF38
:10646000FFFFFFFFFFFFFFFFFFFFFFFFFFFFFFFF3C
:10647000FFFFFFFFFFFFFFFFFFFFFFFFFFFFFFFF2C
:10648000FFFFFFFFFFFFFFFFFFFFFFFFFFFFFFFF1C
:10649000FFFFFFFFFFFFFFFFFFFFFFFFFFFFFFFF0C
:0200000400F00A
:10000000E80300313233340030383335333135359D
:100010003330FFFFFFFFFFFFFFFFFFFFFFFFFFFF8B
:10002000FFFFFFFFFFFFFFFFFFFFFFFFFFFFFFFFE0
:10003000FFFFFFFFFFFFFFFFFFFFFFFFFFFFFFFFD0
:10004000FFFFFFFFFFFFFFFFFFFFFFFFFFFFFFFFC0
:10005000FFFFFFFFFFFFFFFFFFFFFFFFFFFFFFFFB0
:10006000FFFFFFFFFFFFFFFFFFFFFFFFFFFFFFFFA0
:10007000FFFFFFFFFFFFFFFFFFFFFFFFFFFFFFFF90
:10008000FFFFFFFFFFFFFFFFFFFFFFFFFFFFFFFF80
:10009000FFFFFFFFFFFFFFFFFFFFFFFFFFFFFFFF70
:1000A000FFFFFFFFFFFFFFFFFFFFFFFFFFFFFFFF60
:1000B000FFFFFFFFFFFFFFFFFFFFFFFFFFFFFFFF50
:1000C0008C87827D787573716D696766656463621C
:1000D00061605F5E5E5D5D5C5C5B5B5A5A5959595D
:1000E00058585857575756565655555555545454B1
:1000F00054535353535352525252515151515151DF
:020000040030CA
:0E0000000023003C0099800000000FE00F403C
:020000040020DA
:08000000FFFFFFFFFFFFFFFF00
:00000001FF
